:020000040000FA
:0608000078EF38F0120051
:060808009FEF38F0120022
:0608180053EF38F012005E
:06082A00020096710000BF
:10083000F0000000070000007C710000CC00000008
:040840001A0000009A
:0C084400D9CFE6FFE1CFD9FF120EE1266C
:100850000C0EDB6AFE0EDB50050818E0FE0EDB50C6
:10086000060814E0FE0EDB50070810E0FE0EDB5019
:1008700018080CE0FE0EDB50190808E0FE0EDB50F5
:100880001A0804E0FE0EDB502F0803E2000EA0EF72
:100890000DF0FD0EDB50010803E2000EA0EF0DF09D
:1008A000F90EDBCF00F0FA0EDBCF01F0FB0EDBCF51
:1008B00002F0FC0EDBCF03F09A0E326E990E336E0F
:1008C000990E346E3F0E356E00C02DF001C02EF033
:1008D00002C02FF003C030F0E2EC26F0010A01E183
:1008E00026D1F90EDBCF04F0FA0EDBCF05F0FB0EBC
:1008F000DBCF06F0FC0EDBCF07F09A0E326E990EBE
:10090000336E190E346E400E356E04C02DF005C0E6
:100910002EF006C02FF007C030F0E2EC26F0010AFE
:1009200001E105D1F90EDBCF08F0FA0EDBCF09F0BB
:10093000FB0EDBCF0AF0FC0EDBCF0BF09A0E326E13
:10094000990E336E990E346E400E356E08C02DF040
:1009500009C02EF00AC02FF00BC030F0E2EC26F0F8
:10096000010A01E1E4D0F90EDBCF0CF0FA0EDBCF87
:100970000DF0FB0EDBCF0EF0FC0EDBCF0FF09A0E6E
:10098000326E990E336E190E346E410E356E0CC0F8
:100990002DF00DC02EF00EC02FF00FC030F0E2ECA5
:1009A00026F0010A01E1C3D0F90EDBCF10F0FA0EF8
:1009B000DBCF11F0FB0EDBCF12F0FC0EDBCF13F020
:1009C0009A0E326E990E336E990E346E410E356E5C
:1009D00010C02DF011C02EF012C02FF013C030F057
:1009E000E2EC26F0010A01E1A2D0F90EDBCF14F00F
:1009F000FA0EDBCF15F0FB0EDBCF16F0FC0EDBCFD3
:100A000017F09A0E326E990E336E190E346E420E36
:100A1000356E14C02DF015C02EF016C02FF017C083
:100A200030F0E2EC26F0010A01E181D0F90EDBCFD3
:100A300018F0FA0EDBCF19F0FB0EDBCF1AF0FC0E2C
:100A4000DBCF1BF0660E326E660E336E660E346EB2
:100A5000420E356E18C02DF019C02EF01AC02FF0BE
:100A60001BC030F0E2EC26F0010A61E0F90EDBCFAA
:100A70001CF0FA0EDBCF1DF0FB0EDBCF1EF0FC0EE0
:100A8000DBCF1FF09A0E326E990E336E990E346ED4
:100A9000420E356E1CC02DF01DC02EF01EC02FF072
:100AA0001FC030F0E2EC26F0010A41E0F90EDBCF86
:100AB00020F0FA0EDBCF21F0FB0EDBCF22F0FC0E94
:100AC000DBCF23F0326A336AC00E346E420E356ECD
:100AD00020C02DF021C02EF022C02FF023C030F016
:100AE000E2EC26F0010A23E0F90EDBCF24F0FA0E47
:100AF000DBCF25F0FB0EDBCF26F0FC0EDBCF27F0A3
:100B0000660E326E660E336EE60E346E420E356E33
:100B100024C02DF025C02EF026C02FF027C030F0C5
:100B2000E2EC26F0010A03E0000EA0EF0DF0F60E55
:100B3000DB50070807E0F60EDB50080803E0000E64
:100B4000A0EF0DF0F50EDB50020803E2000EA0EF5F
:100B50000DF0FE0EDB500CE0D950F70FE96EFF0EE2
:100B6000DA20EA6EEE50ED1003E0000EA0EF0DF07B
:100B7000EF0EDB501CE0EF0EDB50050818E0EF0E27
:100B8000DB50060814E0EF0EDB50070810E0EF0E14
:100B9000DB5018080CE0EF0EDB50190808E0EF0EF0
:100BA000DB501A0804E0EF0EDB502F0803E2000EC2
:100BB000A0EF0DF0FE0EDB50F36EEF0EDB50F35C9A
:100BC00003E1000EA0EF0DF02D6A2E6A200E2F6EAD
:100BD000410E306EF90EDBCF32F0FA0EDBCF33F080
:100BE000FB0EDBCF34F0FC0EDBCF35F01FEC26F034
:100BF000B3EC26F02EC0DEFF2FC0DDFF020EDB6A55
:100C0000030EDB6A040EDB6A010EF36E050EF3CFF2
:100C1000DBFFFD0EDB5002E1050EDB6AEF0EDB5061
:100C20002F0A01E1EBD3010A01E1D3D3030A01E169
:100C3000BBD3010A01E1A3D3070A01E18BD3010A67
:100C400001E173D3030A01E15BD3010A01E143D35C
:100C50000F0A01E12BD3010A01E113D3030A01E1D9
:100C6000FBD2010A01E1E3D2070A01E1CBD2010A7A
:100C700001E1B3D2030A01E19BD2010A01E183D26F
:100C80003F0A01E16BD2010A01E153D2030A01E1FB
:100C90003BD2010A01E123D2070A01E10BD2020A89
:100CA00001E1F3D1010A01E1DBD10F0A01E1C0D179
:100CB000010A01E1A8D1030A01E190D1010A01E191
:100CC00076D1070A01E15FD1010A01E148D1030AA7
:100CD00001E131D1010A01E11AD11F0A01E103D179
:100CE000010A01E1EAD0030A01E1D1D0010A01E1E0
:100CF000BAD0070A01E1A3D0010A01E18AD0030AB0
:100D000074E0010A5DE00C0A46E0070A2FE0010AE0
:100D100018E0030A01E086D3EF0EB014B06EFD0EAA
:100D20009614966ED9500D0FE96EDACFEAFF8D0E4C
:100D3000EE6E0F0EED6E020EF36E0F0EF3CFDBFFB5
:100D400071D3EF0EB014B06EFE0E9614966ED9509D
:100D50000D0FE96EDACFEAFF8D0EEE6E0F0EED6E1F
:100D6000010EF36E0F0EF3CFDBFF5CD3F00EB71462
:100D7000B76EFE0E9814986ED9500D0FE96EDACF4B
:100D8000EAFF8F0EEE6E0F0EED6E010EF36E0F0E7C
:100D9000F3CFDBFF47D37F0E6B146B6EFD0E981401
:100DA000986ED9500D0FE96EDACFEAFF8F0EEE6E16
:100DB0000F0EED6E020EF36E0F0EF3CFDBFF32D38C
:100DC000DF0EC614C66E7F0E9714976ED9500D0FA6
:100DD000E96EDACFEAFF8E0EEE6E0F0EED6E800E2C
:100DE000F36E0F0EF3CFDBFF1DD30F0EC16EBF0EE0
:100DF0009714976ED9500D0FE96EDACFEAFF8E0E79
:100E0000EE6E0F0EED6E400EF36E0F0EF3CFDBFFA6
:100E100009D3070EB46E0F0EC16EDF0E9714976ED6
:100E2000D9500D0FE96EDACFEAFF8E0EEE6E0F0E7F
:100E3000ED6E200EF36E0F0EF3CFDBFFF3D20F0E2D
:100E4000C16EEF0E9714976ED9500D0FE96EDACF81
:100E5000EAFF8E0EEE6E0F0EED6E100EF36E0F0E9D
:100E6000F3CFDBFFDFD20F0EC16EF70E9714976E34
:100E7000D9500D0FE96EDACFEAFF8E0EEE6E0F0E2F
:100E8000ED6E080EF36E0F0EF3CFDBFFCBD2070E25
:100E9000B46E0F0EC16EFB0E9714976ED9500D0FE6
:100EA000E96EDACFEAFF8E0EEE6E0F0EED6E040ED7
:100EB000F36E0F0EF3CFDBFFB5D2070EB46E0F0E3D
:100EC000C16EFD0E9714976ED9500D0FE96EDACFF3
:100ED000EAFF8E0EEE6E0F0EED6E020EF36E0F0E2B
:100EE000F3CFDBFF9FD20F0EC16EFE0E9714976EED
:100EF000D9500D0FE96EDACFEAFF8E0EEE6E0F0EAF
:100F0000ED6E010EF36E0F0EF3CFDBFF8BD20F0EE3
:100F1000C16EF70E9214926ED9500D0FE96EDACFB2
:100F2000EAFF890EEE6E0F0EED6E080EF36E0F0ED9
:100F3000F3CFDBFF77D20F0EC16EFB0E9214926ED1
:100F4000D9500D0FE96EDACFEAFF890EEE6E0F0E63
:100F5000ED6E040EF36E0F0EF3CFDBFF63D20F0EB8
:100F6000C16EFD0E9214926ED9500D0FE96EDACF5C
:100F7000EAFF890EEE6E0F0EED6E020EF36E0F0E8F
:100F8000F3CFDBFF4FD20F0EC16EFE0E9214926EA6
:100F9000D9500D0FE96EDACFEAFF890EEE6E0F0E13
:100FA000ED6E010EF36E0F0EF3CFDBFF3BD20F0E93
:100FB000C16EEF0ED214D26EDF0E9214926ED95023
:100FC0000D0FE96EDACFEAFF890EEE6E0F0EED6EB1
:100FD000200EF36E0F0EF3CFDBFF24D2DF0ED514FD
:100FE000D56EEF0E9214926ED9500D0FE96EDACFD6
:100FF000EAFF890EEE6E0F0EED6E100EF36E0F0E01
:10100000F3CFDBFF0FD2F70ECD14CD6EFD0E94148F
:10101000946ED9500D0FE96EDACFEAFF8B0EEE6EAB
:101020000F0EED6E020EF36E0F0EF3CFDBFFFAD153
:10103000F50ECD14CD6EFD0EB114B16EFE0E9414EE
:10104000946ED9500D0FE96EDACFEAFF8B0EEE6E7B
:101050000F0EED6E010EF36E0F0EF3CFDBFFE2D13C
:101060007F0EAB14AB6EBF0E9414946ED9500D0F5F
:10107000E96EDACFEAFF8B0EEE6E0F0EED6E400ECC
:10108000F36E0F0EF3CFDBFFCDD17F0EAB14AB6E43
:101090007F0E9414946ED9500D0FE96EDACFEAFFEB
:1010A0008B0EEE6E0F0EED6E800EF36E0F0EF3CF05
:1010B000DBFFB8D1F00EBD14BD6EFB0E9414946E20
:1010C000D9500D0FE96EDACFEAFF8B0EEE6E0F0EE0
:1010D000ED6E040EF36E0F0EF3CFDBFFA3D1DF0E28
:1010E000C614C66EF70E9414946ED9500D0FE96EA7
:1010F000DACFEAFF8B0EEE6E0F0EED6E080EF36E7A
:101100000F0EF3CFDBFF8ED1DF0EC614C66EEF0ECF
:101110009414946ED9500D0FE96EDACFEAFF8B0E5E
:10112000EE6E0F0EED6E100EF36E0F0EF3CFDBFFB3
:1011300079D1DF0EC614C66EDF0E9414946ED950AA
:101140000D0FE96EDACFEAFF8B0EEE6E0F0EED6E2D
:10115000200EF36E0F0EF3CFDBFF64D1F70EF21407
:10116000F26E7F0E9314936ED9500D0FE96EDACFA5
:10117000EAFF8A0EEE6E0F0EED6E800EF36E0F0E0E
:10118000F3CFDBFF4FD1F70EF214F26EBF0E9314C4
:10119000936ED9500D0FE96EDACFEAFF8A0EEE6E2C
:1011A0000F0EED6E400EF36E0F0EF3CFDBFF3AD154
:1011B000F70EF214F26EDF0E9314936ED9500D0FEA
:1011C000E96EDACFEAFF8A0EEE6E0F0EED6E200E9C
:1011D000F36E0F0EF3CFDBFF25D1F70EF214F26E94
:1011E000EF0E9314936ED9500D0FE96EDACFEAFF2C
:1011F0008A0EEE6E0F0EED6E100EF36E0F0EF3CF25
:10120000DBFF10D1DF0EF014F06EF70E9314936E27
:10121000D9500D0FE96EDACFEAFF8A0EEE6E0F0E8F
:10122000ED6E080EF36E0F0EF3CFDBFFFBD0EF0E6B
:10123000F014F06EFB0E9314936ED9500D0FE96EFF
:10124000DACFEAFF8A0EEE6E0F0EED6E040EF36E2D
:101250000F0EF3CFDBFFE6D0F70EF014F06EFD0EAD
:101260009314936ED9500D0FE96EDACFEAFF8A0E10
:10127000EE6E0F0EED6E020EF36E0F0EF3CFDBFF70
:10128000D1D0EF0EF214F26EFE0E9314936ED9507D
:101290000D0FE96EDACFEAFF8A0EEE6E0F0EED6EDD
:1012A000010EF36E0F0EF3CFDBFFBCD0EF0EB014C8
:1012B000B06E7F0E9514956ED9500D0FE96EDACF92
:1012C000EAFF8C0EEE6E0F0EED6E800EF36E0F0EBB
:1012D000F3CFDBFFA7D0EF0EB014B06EBF0E9514A6
:1012E000956ED9500D0FE96EDACFEAFF8C0EEE6ED7
:1012F0000F0EED6E400EF36E0F0EF3CFDBFF92D0AC
:10130000EF0EB014B06EDF0E9514956ED9500D0F20
:10131000E96EDACFEAFF8C0EEE6E0F0EED6E200E48
:10132000F36E0F0EF3CFDBFF7DD0EF0EB014B06E77
:10133000EF0E9514956ED9500D0FE96EDACFEAFFD6
:101340008C0EEE6E0F0EED6E100EF36E0F0EF3CFD1
:10135000DBFF68D0EF0EB014B06EF70E9514956EEB
:10136000D9500D0FE96EDACFEAFF8C0EEE6E0F0E3C
:10137000ED6E080EF36E0F0EF3CFDBFF53D0EF0EC2
:10138000B014B06EFB0E9514956ED9500D0FE96E2A
:10139000DACFEAFF8C0EEE6E0F0EED6E040EF36EDA
:1013A0000F0EF3CFDBFF3ED0EF0EB014B06EFD0E8C
:1013B0009514956ED9500D0FE96EDACFEAFF8C0EB9
:1013C000EE6E0F0EED6E020EF36E0F0EF3CFDBFF1F
:1013D00029D0EF0EB014B06EFE0E9514956ED95054
:1013E0000D0FE96EDACFEAFF8C0EEE6E0F0EED6E8A
:1013F000010EF36E0F0EF3CFDBFF14D0EF0EB0141F
:10140000B06EFB0E9614966ED9500D0FE96EDACFC2
:10141000EAFF8D0EEE6E0F0EED6E040EF36E0F0EE4
:10142000F3CFDBFF0F0EDB1CE76E100EE7CFDBFF09
:101430000F0EDBCFE6FF0D0EDBCFE9FF0E0EDBCF8D
:10144000EAFFEF50E552E710E76E0F0EE7CFDBFF44
:10145000100EDBCFE6FF0D0EDBCFE9FF0E0EDBCF6C
:10146000EAFFEF50E552E714E76E100EE7CFDBFF1F
:101470000D0EDBCFE9FF0E0EDBCFEAFF0F0EDBCF49
:10148000EFFF000EDBCF2EF0010EDBCF2FF0800E32
:101490002E1802E1040E2F1871E0C00E2E1802E182
:1014A000030E2F1865E02E5002E1030E2F185AE0AC
:1014B000400E2E1802E1020E2F184EE0800E2E185C
:1014C00002E1010E2F1842E0C00E2E1801E12F504C
:1014D00037E0600E2E1801E12F502CE0300E2E1850
:1014E00001E12F5021E0180E2E1801E12F5011E0DC
:1014F0000C0E2E1801E12F5001E045D03D0EF36E89
:101500000B0EF3CFDBFF030EF36E0C0EF3CFDBFFFE
:101510003AD09E0EF36E0B0EF3CFDBFF010EF36E8F
:101520000C0EF3CFDBFF2FD0CE0EF36E0B0EF3CFEE
:10153000DBFF29D0660EF36E0B0EF3CFDBFF23D05B
:10154000320EF36E0B0EF3CFDBFF1DD0170EF36ED2
:101550000B0EF3CFDBFF17D00F0EF36E0B0EF3CF96
:10156000DBFF11D00A0EF36E0B0EF3CFDBFF0BD0B7
:10157000080EF36E0B0EF3CFDBFF05D0060EF36EF5
:101580000B0EF3CFDBFFFE0EDB501CE0D950F30F48
:10159000E96EFF0EDA20EA6EEE50ED1013E1FE0E5A
:1015A000DBCFE6FF92EC2CF0E552E76E0A0EE7CFB8
:1015B000DBFF050EDB50F36E0A0EDB50F35C01E13E
:1015C00001D0EDD7FE0EDB503DE0D950F30FE96EB0
:1015D000FF0EDA20EA6EEE50ED1034E0020EDB6A08
:1015E000030EDB6ABAEC37F0FE0EDBCFE6FF92ECBF
:1015F0002CF0E552E76E0A0EE7CFDBFF050EDB505D
:10160000F36E0A0EDB50F35C01E11CD0C1EC37F045
:10161000000917E0020EDB2A030E01E3DB2A020EAB
:10162000DBCF00F0030EDBCF01F0F30EDB50001830
:1016300003E1F40EDB50011802E1020E81D2BAEC94
:1016400037F0D2D7040EDB50E76EF10EDBCFE9FFA7
:10165000F20EDBCFEAFFE750E926000EEA22060E83
:10166000EFCFDBFF040EDB2AF60EDB50070807E1A5
:10167000060EDB507F0BE76E060EE7CFDBFFF50EA5
:10168000DB5053E0090EDB6A080EDB6AF60EDB5016
:10169000F36E080EDBCFF4FFF350F45C1CE2D9507C
:1016A000080FE96EDACFEAFF060EDB50EFCFE7FF57
:1016B000E75204E0E8427F0BE706FCE1010B006E15
:1016C000090EDBCFE7FF0050E726090EE7CFDBFF6F
:1016D000080EDB2ADBD7070EDB6AF50EDB040AE116
:1016E000090EDB50010B06E0010EF36E070EF3CF7F
:1016F000DBFF0DD0F50EDB50020809E1090EDB50CF
:10170000010B05E1010EF36E070EF3CFDBFFF60EC2
:10171000DB5007080AE1070EDB5007E0060EDB503E
:101720008009E76E060EE7CFDBFFFE0EDB5013E10C
:10173000D950F70FE96EFF0EDA20EA6EEE50ED1089
:101740000AE0F70EDBCFE6FFF80EDBCFE6FFD0ECCA
:1017500037F0E552E55204000D0EDBCFE9FF0E0E27
:10176000DBCFEAFF100EDBCFEFFF110EDB6A0C0EB2
:10177000DB50F36E110EDBCFF4FFF350F45C07E2A5
:10178000E66894EC38F0E552110EDB2AF0D70B0E28
:10179000DBCFE6FF94EC38F0E552060EDBA009D073
:1017A0000D0EDBCFE9FF0E0EDBCFEAFF0F0EDBCF16
:1017B000EFFF110EDB6A0C0EDB50F36E110EDBCF68
:1017C000F4FFF350F45C07E2E66894EC38F0E5527D
:1017D000110EDB2AF0D70B0EDBCFE6FF94EC38F0CE
:1017E000E552060EDBA20AD00D0EDBCFE9FF0E0E8E
:1017F000DBCFEAFF0F0EDBCFEFFF09D00D0EDBCF03
:10180000E9FF0E0EDBCFEAFF100EDBCFEFFF110E6C
:10181000DB6A0C0EDB50F36E110EDBCFF4FFF350DE
:10182000F45C07E2E66894EC38F0E552110EDB2A2E
:10183000F0D70B0EDBCFE6FF94EC38F0E552060E46
:10184000DBA40AD00D0EDBCFE9FF0E0EDBCFEAFFE3
:101850000F0EDBCFEFFF09D00D0EDBCFE9FF0E0E31
:10186000DBCFEAFF100EDBCFEFFF110EDB6A0C0EB1
:10187000DB50F36E110EDBCFF4FFF350F45C07E2A4
:10188000E66894EC38F0E552110EDB2AF0D70B0E27
:10189000DBCFE6FF94EC38F0E552060EDBA60AD06B
:1018A0000D0EDBCFE9FF0E0EDBCFEAFF0F0EDBCF15
:1018B000EFFF09D00D0EDBCFE9FF0E0EDBCFEAFF05
:1018C000100EDBCFEFFF110EDB6A0C0EDB50F36E58
:1018D000110EDBCFF4FFF350F45C07E2E66894EC02
:1018E00038F0E552110EDB2AF0D70B0EDBCFE6FF06
:1018F00094EC38F0E552060EDBA80AD00D0EDBCFD3
:10190000E9FF0E0EDBCFEAFF0F0EDBCFEFFF09D0B2
:101910000D0EDBCFE9FF0E0EDBCFEAFF100EDBCFA3
:10192000EFFF110EDB6A0C0EDB50F36E110EDBCFF6
:10193000F4FFF350F45C07E2E66894EC38F0E5520B
:10194000110EDB2AF0D70B0EDBCFE6FF94EC38F05C
:10195000E552060EDBAA0AD00D0EDBCFE9FF0E0E14
:10196000DBCFEAFF0F0EDBCFEFFF09D00D0EDBCF91
:10197000E9FF0E0EDBCFEAFF100EDBCFEFFF110EFB
:10198000DB6A0C0EDB50F36E110EDBCFF4FFF3506D
:10199000F45C07E2E66894EC38F0E552110EDB2ABD
:1019A000F0D70B0EDBCFE6FF94EC38F0E552060ED5
:1019B000DBAC0AD00D0EDBCFE9FF0E0EDBCFEAFF6A
:1019C0000F0EDBCFEFFF09D00D0EDBCFE9FF0E0EC0
:1019D000DBCFEAFF100EDBCFEFFF110EDB6A0C0E40
:1019E000DB50F36E110EDBCFF4FFF350F45C07E233
:1019F000E66894EC38F0E552110EDB2AF0D70B0EB6
:101A0000DBCFE6FF94EC38F0E552F60EDB50080829
:101A100003E0F50EDB502EE0060EDBAE0AD00D0E15
:101A2000DBCFE9FF0E0EDBCFEAFF0F0EDBCFEFFFC0
:101A300009D00D0EDBCFE9FF0E0EDBCFEAFF100E53
:101A4000DBCFEFFF110EDB6A0C0EDB50F36E110ED5
:101A5000DBCFF4FFF350F45C07E2E66894EC38F077
:101A6000E552110EDB2AF0D70B0EDBCFE6FF94EC2C
:101A700038F0E552F60EDB50080831E1F50EDB5088
:101A80002EE0070EDB500AE00D0EDBCFE9FF0E0E55
:101A9000DBCFEAFF0F0EDBCFEFFF09D00D0EDBCF60
:101AA000E9FF0E0EDBCFEAFF100EDBCFEFFF110ECA
:101AB000DB6A0C0EDB50F36E110EDBCFF4FFF3503C
:101AC000F45C07E2E66894EC38F0E552110EDB2A8C
:101AD000F0D70B0EDBCFE6FF94EC38F0E5520D0E9D
:101AE000DBCFE9FF0E0EDBCFEAFF0F0EDBCFEFFF00
:101AF000110EDB6A0C0EDB50F36E110EDBCFF4FF20
:101B0000F350F45C07E2E66894EC38F0E552110E0D
:101B1000DB2AF0D70B0EDBCFE6FF94EC38F0E55272
:101B2000F00EDB50F36E040EDB50F35C06E0F00EBB
:101B3000DB5005E1060EDB5002E1010E01D023D59A
:101B4000006E120EE15C02E2E16AE552E16E0050C5
:081B5000E552E7CFD9FF1200B6
:081B5800D9CFE6FFE1CFD9FF70
:101B6000FE0EDBCFA2F0FD0EDBCFA3F0FB0EDBCF32
:101B700000F0FC0EDBCF01F001C000F0016A005064
:101B80000001A46FFF0EE76EFB0EDBCF00F0FC0E32
:101B9000DBCF01F0E7500016016A00C0A5F0A66B8C
:101BA000D70EE66E000EE66E050EE66EA20EE66E2F
:101BB000000EE66E96EC36F0006E050EE15E00500B
:101BC000000902E10001D66BE552E7CFD9FF120010
:101BD000D9CFE6FFE1CFD9FF060EE126040EE66E6F
:101BE000E66AE66ABA0EE66E000EE66E4EEC34F079
:101BF000006E050EE15E0050040EE66EE66AE66ACF
:101C0000BE0EE66E000EE66E4EEC34F0006E050E73
:101C1000E15E0050040EE66EE66AE66AC60EE66E07
:101C2000000EE66E4EEC34F0006E050EE15E0050E4
:101C3000040EE66EE66AE66AC20EE66E000EE66E18
:101C40004EEC34F0006E050EE15E0050040EE66EC0
:101C5000E66AE66AB60EE66E000EE66E4EEC34F00C
:101C6000006E050EE15E0050040EE66EE66AE66A5E
:101C7000B20EE66E000EE66E4EEC34F0006E050E0F
:101C8000E15E0050010EE66EDAC0E6FF21EC28F0BE
:101C9000E552E552010EE66EDBC0E6FF21EC28F0CE
:101CA000E552E552E80EE66E030EE66ED0EC37F034
:101CB000E552E552E66ADBC0E6FF21EC28F0E5528A
:101CC000E552F40EE66E010EE66ED0EC37F0E5520A
:101CD000E552010EE66EDBC0E6FF21EC28F0E5528E
:101CE000E552E80EE66E030EE66ED0EC37F0E552F4
:101CF000E5520001010EB06F0001010ED66F000E1B
:101D0000E66EE66AD9CFE6FFDACFE6FFD70EE66EDB
:101D1000000EE66E000EE66EE66A050EE66ED3EC89
:101D200020F0006E090EE15E0050000901E1E4D7E9
:101D30000001B051000808E2010EE66EDCC0E6FFCB
:101D400021EC28F0E552E5520001AE6B050EAE5DC8
:101D500025E2D70EE66E000EE66E010EE66EA70EC9
:101D6000E66E000EE66E880EE66E130EE66EDFEC93
:101D700035F0006E070EE15E0050010801E00ED064
:101D80000001AE51EA6AD10FE96E000EEA22EF506F
:101D9000A75D02E1AE2B01D0AE6BD8D7050E0001D6
:101DA000AE5D15E2000EE66EE66AE66EE66AD70EF6
:101DB000E66E000EE66E000EE66EE66A0A0EE66E4F
:101DC000D3EC20F0006E090EE15E005095D7D70EDF
:101DD000E66E000EE66E050EE66ECC0EE66E000EAA
:101DE000E66E96EC36F0006E050EE15E00500009DE
:101DF00015E1000EE66EE66AE66EE66AD70EE66E5E
:101E0000000EE66E000EE66EE66A0A0EE66ED3EC93
:101E100020F0006E090EE15E00506ED70001B16B3C
:101E200004012C6B0001D65102E1A1EF14F0000176
:101E3000B05100080CE2B051B02B0B0808E2DCC036
:101E4000E6FF7FEC2EF0E5520001010EB06FD70ED9
:101E5000E66E000EE66E050EE66EA70EE66E000E4E
:101E6000E66E0F0EE66EE66ADFEC35F0006E070EEA
:101E7000E15E0050010801E0EBD10001B16BA75118
:101E800001E1E2D10B0A01E10FD1070A01E10CD116
:101E9000010A01E109D1040A01E1D7D0010A01E1F7
:101EA000C2D00F0A01E190D0020A01E17ED0010AFE
:101EB0004CE0070A35E0010A1BE0030A01E0C7D144
:101EC000A8C000F000C001F0006AA9510001001094
:101ED000DF6F01C0E0F0AAC000F000C001F0006AAE
:101EE0000001AB5100010010DD6F01C0DEF0AFD189
:101EF000A8C000F000C001F0006AA9510001001064
:101F0000E16F01C0E2F0AAC000F000C001F0006A79
:101F10000001AB5100010010E36F01C0E4F097D164
:101F2000D70EE66E000EE66E050EE66EA70EE66EA6
:101F3000000EE66E96EC36F0006E050EE15E005087
:101F4000000902E10001D66B82D1AA51320DF3CF14
:101F500004F0F4CF05F004C02EF005C02FF020EC03
:101F600025F02DC000F02EC001F02FC002F030C0CF
:101F700003F000C0E6FF01C0E6FF02C0E6FF03C0B9
:101F8000E6FF0001A951320DF3CF06F0F4CF07F0C0
:101F900006C0E6FF07C0E6FFA8C0E6FFB1EC2FF0E1
:101FA000086E070EE15E085052D1A8510AE0E66AB9
:101FB000DCC0E6FF21EC28F0E552E5520001B06BF1
:101FC00002D0010EB06F43D1040EE66EE66AA80E91
:101FD000E66E000EE66EBA0EE66E000EE66E00ECE1
:101FE00034F0006E060EE15E00500001AE6B040E90
:101FF000AE5D18E2AE51EA6AA70FE96E000EEA2262
:10200000EF500DE0E66AAE51EA6AA70FE96E000EE6
:10201000EA22EF50E66E21EC28F0E552E55200018D
:10202000AE2BE5D714D1040EE66EE66AA80EE66E76
:10203000000EE66EBE0EE66E000EE66E00EC34F0AC
:10204000006E060EE15E005002D1040EE66EE66AF6
:10205000A80EE66E000EE66EB60EE66E000EE66E9A
:1020600000EC34F0006E060EE15E00500001AE6B35
:10207000040EAE5D18E2AE51EA6AA70FE96E000EDB
:10208000EA22EF500DE0E66AAE51EA6AA70FE96E68
:10209000000EEA22EF50E66E21EC28F0E552E55200
:1020A0000001AE2BE5D7D3D0A8C0AFF0AE6B0401D2
:1020B0002C510001AE5D0BE2AE51EA6A000FE96EF1
:1020C000030EEA22EF50AF5D02E0AE2BF0D70B0E0D
:1020D000A75D18E104012C510001AE5D12E304017B
:1020E0002C51EA6A000FE96E030EEA22AFC0EFFF3F
:1020F0002C51EA6AFA0FE96E030EEA22A9C0EFFF3B
:102100002C2BA1D00C0EA75D56E104012C5100012F
:10211000AE5D50E204012C072C5100084BE22C511B
:10212000EA6A000FE96E030EEA22EF50E66E000144
:10213000AE51EA6A000FE96E030EEA22E552E7505B
:10214000EF6E04012C51EA6AFA0FE96E030EEA22DF
:10215000EF50E66E0001AE51EA6AFA0FE96E030E27
:10216000EA22E552E750EF6E04012C51040DF3CF43
:10217000E9FFF4CFEAFF320EE926030EEA22EECFA2
:1021800000F0EECF01F0EECF02F0EFCF03F0000150
:10219000AE51040DF3CFE9FFF4CFEAFF320EE9268A
:1021A000030EEA2200C0EEFF01C0EEFF02C0EEFF08
:1021B00003C0EEFF48D004012C510001AE5D43E2A4
:1021C000AAC000F000C001F0006AAB510010AC6F73
:1021D00001C0ADF0ACC02EF0ADC02FF020EC25F06A
:1021E0002DC004F02EC005F02FC006F030C007F05F
:1021F000326A336A7A0E346E440E356E04C02DF0A6
:1022000005C02EF006C02FF007C030F0CCEC25F052
:102210002DC000F02EC001F02FC002F030C003F03E
:102220000001AE51040DF3CFE9FFF4CFEAFF320E07
:10223000E926030EEA2200C0EEFF01C0EEFF02C055
:10224000EEFF03C0EEFF03D00001D66B00D00FD02D
:102250000001B12BB151006E016AD890015004E623
:10226000C80E005C000E015802E30001D66B010E9F
:10227000E66EE66EDFC0E6FFE0C0E6FF100EE66E3B
:10228000BBEC34F0006E050EE15E0050010EE66E10
:10229000E66EDDC0E6FFDEC0E6FF110EE66EBBECCB
:1022A00034F0006E050EE15E0050010EE66EE66E43
:1022B000E1C0E6FFE2C0E6FF120EE66EBBEC34F0D2
:1022C000006E050EE15E0050010EE66EE66EE3C0A4
:1022D000E6FFE4C0E6FF130EE66EBBEC34F0006EE2
:1022E000050EE15E00500001CA6BAE6B040EAE5DE0
:1022F0006EE2AE51EA6ABA0FE96E000EEA22EF50C2
:1023000064E0AE51EA6ABE0FE96E000EEA22EF50B9
:102310005CE0AE51EA6AC20FE96E000EEA22EF50AD
:102320001CE10F0EE66EE66A020EE66EAE51EA6A38
:10233000BA0FE96E000EEA22EF50E66EB7EC30F00D
:10234000E552E552E552E5520001AE51EA6AC20F8C
:10235000E96E000EEA22EF2A38D0AE51EA6AC20FC7
:10236000E96E000EEA22EF50280828E2AE51EA6A30
:10237000BE0FE96E000EEA22EF50E66E92EC2CF0F2
:10238000E5520001AF6FAE51EA6AC60FE96E000E6A
:10239000EA22EF50AF5D0AE0AE51EA6AC60FE96E7D
:1023A000000EEA22AFC0EFFF010ECA6FAE51EA6A1B
:1023B000C20FE96E000EEA22EF6A07D0AE51EA6A58
:1023C000C20FE96E000EEA22EF2AAE2B8FD7CA5158
:1023D00027E0070EA76F040EE66EE66AC60EE66EED
:1023E000000EE66EA80EE66E000EE66E00EC34F00F
:1023F000006E060EE15E0050D70EE66E000EE66E31
:10240000050EE66EA70EE66E000EE66E96EC36F052
:10241000006E050EE15E0050000902E10001D66B7E
:102420000001E551EA6AB60FE96E000EEA22EFCF2D
:10243000CBF00001CA6BCB5101E1C4D0E66ACBC03E
:10244000E6FF21EC28F0E552E552020EE66EE66A60
:1024500093EC37F0E552E552010EE66EE66AE66E61
:10246000E66ACBC0E6FFBBEC34F0006E050EE15E21
:102470000050020EE66EE66A93EC37F0E552E55244
:10248000260EE66EE66A010EE66ECBC0E6FF7FEC36
:1024900032F0E552E552E552E552F3CFACF0F4CF1D
:1024A000ADF00001AC51AD1174E00C6AE00E0D6EA0
:1024B000530E0E6E460E0F6EACC02EF0ADC02FF058
:1024C00020EC25F02DC010F02EC011F02FC012F01E
:1024D00030C013F010C032F011C033F012C034F02D
:1024E00013C035F00CC02DF00DC02EF00EC02FF033
:1024F0000FC030F01FEC26F02DC008F02EC009F000
:102500002FC00AF030C00BF0950E326EBF0E336E46
:10251000560E346E350E356E08C02DF009C02EF003
:102520000AC02FF00BC030F01FEC26F02DC004F0D5
:102530002EC005F02FC006F030C007F0326A336AB3
:10254000346A400E356E04C02DF005C02EF006C072
:102550002FF007C030F0CCEC25F02DC000F02EC0DD
:1025600001F02FC002F030C003F0326A336A400E2F
:10257000346E356E00C02DF001C02EF002C02FF079
:1025800003C030F035EC25F08CEC26F02FC0AFF016
:1025900002D0F00EAF6F0001E551EA6AB20FE96EAA
:1025A000000EEA22EF500001AF5D0CE00001E551A2
:1025B000EA6AB20FE96E000EEA22AFC0EFFF000137
:1025C000010ECA6FCA5127E0090EA76F040EE66E0E
:1025D000E66AB20EE66E000EE66EA80EE66E000E1D
:1025E000E66E00EC34F0006E060EE15E0050D70E91
:1025F000E66E000EE66E050EE66EA70EE66E000EA7
:10260000E66E96EC36F0006E050EE15E00500009B5
:1026100002E10001D66B0001E52B040EE55D01E34C
:10262000E56B0001AE6B04012C510001AE5D01E3CE
:1026300086D1AE51EA6AFA0FE96E030EEA22EF5034
:10264000040A01E158D1070A01E1B0D0010A01E111
:1026500077D0030A01E070D1AE51EA6A000FE96E4B
:10266000030EEA22EF50E66E92EC2CF0E5520001E8
:10267000AF6FAFC02FF00FEC25F02DC000F02EC0D3
:1026800001F02FC002F030C003F00001AE51040D84
:10269000F3CFE9FFF4CFEAFF320EE926030EEA2278
:1026A000EECF04F0EECF05F0EECF06F0EFCF07F05F
:1026B00004C032F005C033F006C034F007C035F076
:1026C00000C02DF001C02EF002C02FF003C030F08A
:1026D000E2EC26F0010A33E00001AF51E66EE66A53
:1026E000AE51EA6A000FE96E030EEA22EF50E66E81
:1026F0000B0EE66EACEC0DF0E552E552E552E552FC
:10270000AFC02FF00FEC25F02DC000F02EC001F06F
:102710002FC002F030C003F00001AE51040DF3CF22
:10272000E9FFF4CFEAFF320EE926030EEA2200C0E9
:10273000EEFF01C0EEFF02C0EEFF03C0EEFFFCD0D3
:10274000AE51040DF3CFE9FFF4CFEAFF320EE926D4
:10275000030EEA22EECF00F0EECF01F0EECF02F052
:10276000EFCF03F0326A336A346A356A00C02DF065
:1027700001C02EF002C02FF003C030F0E9EC26F0CB
:10278000010A02E1010E01D0000EE66E0001AE5119
:10279000EA6A000FE96E030EEA22EF50E66E21ECC2
:1027A00028F0E552E5520001AF6FC6D0E66AE66A4E
:1027B000A00EE66E400EE66EE66AE66AE66AE66A35
:1027C000E66A010EE66EAE51EA6A000FE96E030E8C
:1027D000EA22EF50E66E8FEC2AF0046E0B0EE15EFB
:1027E00004502CC000F02DC001F02EC002F02FC00C
:1027F00003F0326A336A7A0E346E440E356E00C0CE
:102800002DF001C02EF002C02FF003C030F01FECFD
:1028100026F0B3EC26F02EC0ACF02FC0ADF0ACC06B
:102820002EF0ADC02FF020EC25F02DC000F02EC012
:1028300001F02FC002F030C003F00001AE51040DD2
:10284000F3CFE9FFF4CFEAFF320EE926030EEA22C6
:10285000EECF04F0EECF05F0EECF06F0EFCF07F0AD
:1028600004C032F005C033F006C034F007C035F0C4
:1028700000C02DF001C02EF002C02FF003C030F0D8
:10288000E2EC26F0010A36E0ACC0E6FFADC0E6FFA0
:102890000001AE51EA6A000FE96E030EEA22EF5022
:1028A000E66E0B0EE66EACEC0DF0E552E552E5522D
:1028B000E552ACC02EF0ADC02FF020EC25F02DC0BD
:1028C00000F02EC001F02FC002F030C003F0000174
:1028D000AE51040DF3CFE9FFF4CFEAFF320EE92643
:1028E000030EEA2200C0EEFF01C0EEFF02C0EEFFC1
:1028F00003C0EEFF21D0AE51040DF3CFE9FFF4CFBA
:10290000EAFF320EE926030EEA22EECFE6FFEECF13
:10291000E6FFEECFE6FFEFCFE6FFAE51EA6A000F2B
:10292000E96E030EEA22EF50E66EB0EC31F0006E75
:10293000050EE15E005000D00001AE2B74D612EF00
:102940000FF0000EE66EE66AE66EE66AD70EE66EF9
:10295000000EE66E000EE66EE66A0A0EE66ED3EC38
:1029600020F0006E090EE15E00507CEF0EF0060EC6
:10297000E15C02E2E16AE552E16EE552E7CFD9FFA0
:02298000120043
:0E298200FDEC19F0FB0EDBCFF3FFDB06F3508C
:1029900000090AE04BEC1AF0FA0EB6EC1AF0F3E17B
:1029A000011CF1E1010E01D0000E2CEF1AF0FDEC3C
:1029B00019F03B0EE12402E3E168E652E16E010EFC
:1029C000DB6A020EDB6AF90EDBCFF6FFFA0EDBCF15
:1029D000F7FFFB0EDBCFF8FF0800F550DF6EDF508E
:1029E00002E150EF19F0250EDF5C02E043EF19F031
:1029F000030EDB6A040EDB6A050EDB6A060EDB6A79
:102A0000070EDB6A65EC19F02D0EDF5C0CE02B0E77
:102A1000DF5C09E0200EDF5C06E0230EDF5C03E0F4
:102A2000300EDF5C1AE1DF50300A14E0130A0FE0C9
:102A3000030A0AE00B0A05E0060AE4E1030EDB8064
:102A4000E1D7030EDB82DED7030EDB84DBD7030E78
:102A5000DB86D8D7030EDB88D5D72A0EDF5C1BE1D7
:102A600061EC19F0AFEC19F010E0030EDB802E687A
:102A70002F68130EDBCF33F0140EDBCF34F0F4EC01
:102A800027F0040E2CC0DBFF03D0130E98EC19F0D6
:102A900065EC19F00BD0090EDB6A06EC1AF003E0C6
:102AA0007AEC1AF0FAD7090E98EC19F0030EDBB0A5
:102AB000DB982E0EDF5C1BE165EC19F02A0EDF5C63
:102AC0000BE161EC19F0AFEC19F003E1130EEAEC45
:102AD00019F065EC19F00BD0090EDB6A06EC1AF060
:102AE00003E07AEC1AF0FAD7090EEAEC19F0680E56
:102AF000DF5C07E165EC19F0680EDF5C1DE1030E99
:102B000018D0740EDF5C17E07A0EDF5C14E0480E1C
:102B1000DF5C06E0540EDF5C03E05A0EDF5C02E18E
:102B2000020E07D06C0EDF5C03E06A0EDF5C04E18E
:102B3000010E3DEC1AF0C9DBDF506E0A01E17FD3D4
:102B40001E0A01E192D1200A01E18FD13F0A01E181
:102B500049D11A0A01E146D10D0A01E143D1200A07
:102B600001E140D13A0A01E13DD1200A01E13AD127
:102B7000260A01E135D10D0A01E132D11A0A01E13B
:102B8000D9D0200A4AE0300A1FE0460A0EE0250AA2
:102B900001E083D3D950F90FE96EFF0EDA20EA6E17
:102BA000010EEE5E000EEE5AEE5A4BEC1AF0250EB8
:102BB000E66E95DB03E1011C01E169D347EC1AF0F5
:102BC00001E26BD3DB2A69D3080EDB6A040EDB500B
:102BD000010806E2040EDB040FEC1AF0DB508BDB7D
:102BE000080EDB5009E0030EDB50010B05E172DB40
:102BF00001E04DD3080EDB6A64DBEFCFDFFFBFECF3
:102C00001AF003E1011C01E142D347EC1AF001E3A1
:102C1000DB2A60DB01E141D33AD3070EDB50020827
:102C20000FE18BEC1AF0030E52EC1AF00E0EEECF01
:102C3000DBFF0F0EEECFDBFF100EEECFDBFF20D061
:102C4000F70EDBCF03F0F80EDBCF04F0020E035ECD
:102C5000000E045AF70E03C0DBFFF80E04C0DBFFC2
:102C600003C0E9FF04C0EAFF42EC1AF0026A0E0E4C
:102C700000C0DBFF0F0E01C0DBFF100E02C0DBFF48
:102C80000E0EDBCFE6FF0F0EDBCFE6FF100EDBCF25
:102C9000E6FF96EC34F0E552E552E552130E2DC0F6
:102CA000DBFF140E2EC0DBFF060EDB5005E0130E1B
:102CB00086EC1AF001E26ADBAAEC1AF002E2130ECB
:102CC00037DB6DEC1AF006E0040E86EC1AF002E237
:102CD000050E2EDB030EDBB005D0FCDA01E0D7D207
:102CE000080EDB6A090EDB6A0E0EDBCFF6FF0F0E55
:102CF000DBCFF7FF100EDBCFF8FF0800F550DF6EDB
:102D0000DF5014E0B0EC1AF011E2BFEC1AF003E16E
:102D1000011C01E1BCD2BBDB01E3DB2A090EDB2A8B
:102D2000D9500E0FE96E000ECBDBE7D7D3DA01E105
:102D3000B4D2ADD2C6DA110EEECFDBFF120EEDCF5C
:102D4000DBFF110EDBCFE6FF120EDBCFE6FF88ECD8
:102D500034F0E552E552130EF3CFDBFF140EF4CF3F
:102D6000DBFF060EDB5004E0130ED0DB01E20EDBCE
:102D7000AAEC1AF002E2130EDBDAAFDB05E0040E78
:102D8000C5DB02E2050ED4DA030EDBB005D0A2DA11
:102D900001E07DD2080EDB6A090EDB6A110EDBCF83
:102DA000E9FF120EDBCFEAFFEFCFDFFFDF5014E0C9
:102DB000D7DB12E2E4DB03E1011C01E168D267DB4F
:102DC00001E3DB2A090EDB2A110EDB2ADBCFE9FF48
:102DD000120EE8E3DB2AE6D77DDA01E15ED257D2B4
:102DE000030EDB8E070EDB0410E195DB040E5ADBCD
:102DF0000A0EEECFDBFF0B0EEECFDBFF0C0EEECF9D
:102E0000DBFF0D0EEECFDBFF6CD0070EDB500308AF
:102E10002CE1030EDBAE0DD0B2DA020E76DAEFCF84
:102E200000F0016A026A036A00AE39D001680268E4
:102E300035D0F70EDBCF01F0F80EDBCF02F0020E3B
:102E4000015E000E025AF70E01C0DBFFF80E02C051
:102E5000DBFF01C0E9FF02C0EAFFEFCF00F00A0E7E
:102E600000C0DBFF0B0EDB6A38D0070EDB50020818
:102E700009E1030EDBAE04D059DB02AE10D00ED058
:102E800055DB0DD0030EDBAE12D079DA020E3DDA3F
:102E9000F9DA026A036A01AE02D002680368E2DA74
:102EA0000C0E02C0DBFF0D0E03C0DBFF1AD0F70EC5
:102EB000DBCF02F0F80EDBCF03F0020E025E000E55
:102EC000035AF70E02C0DBFFF80E03C0DBFF02C09F
:102ED000E9FF03C0EAFFD6DAC5DA0C0EDB6A0D0E95
:102EE000DB6A060EDB5005E1010EF36E050EF3CF33
:102EF000DBFF150EDB6A160EDB6AD950370F006E4A
:102F0000000EDA20016E390E00C0DBFF3A0E01C060
:102F1000DBFF380EDB6A080EDB6A0A0EAEDADF5022
:102F2000780A12E0200A10E0280A0CE0200A0AE0E1
:102F30003F0A06E00D0A02E0200A08E1020E05D071
:102F4000080E03D0080EDF26100E97DA030EDBBE44
:102F500002D0DB92DB94DB50800B24E08ADAD8903D
:102F6000030EEB50000A08E6000EEE5C000EEE5871
:102F7000000EEE58000EEE5815E213DA3168326892
:102F800033683468F7EC37F00A0E28C0DBFF0B0E0D
:102F900029C0DBFF0C0E2AC0DBFF0D0E2BC0DBFFB0
:102FA0002D0E08D0030EDBA202D02B0E03D0DBA423
:102FB00008D0200EF36E170EF3CFDBFF150EDB2AC1
:102FC00002D0170EDB6A050EDB5003E1B7D901E131
:102FD00089D0500E006E710E016E000E026E070E4B
:102FE000DBCF03F0046A056A066A03C031F004C04F
:102FF00032F005C033F006C034F0D3D92FEC38F0EE
:1030000000502824F36E01502920F46E02502A202B
:10301000F86EF4CFF7FFF3CFF6FF0800090EF5CFF7
:10302000DBFF580EDF5C0FE1610EF36E090E7BD9FA
:103030000AE3200E006E090EDBCFE7FF0050E75ECB
:10304000090EE7CFDBFF070EDBCF00F0016A026A53
:10305000036A0FDA00C031F001C032F002C033F071
:1030600003C034F0EECF2CF0EECF2DF0EECF2EF0EB
:10307000EFCF2FF02FEC38F02FC0EDFF2EC0EDFF7B
:103080002DC0EDFF2CC0EFFF390EDBCFE9FFDB06D3
:103090003A0EDBCFEAFF01E2DB06090EDBCFEFFFE2
:1030A000150EDB2A4BD995E1030EDBA61DD06F0E62
:1030B000DF5C06E1C1D918E3150EDB285BDA14D01A
:1030C000780EDF5C09E0580EDF5C06E0620EDF5C24
:1030D00003E0420EDF5C08E1020EF36E160EF3CF42
:1030E000DBFF02D0150EDB6A030EDB50100B0EE087
:1030F000040EDBCF00F0050EDB50D880005406E252
:10310000060EDB5003E1040EDB5034DA95D90AE2F7
:10311000050EDBCFE7FF150EDB50E75E050EE7CFB0
:10312000DBFF02D0050EDB6A040EDBCF00F0160ECB
:1031300045D9D880005414E2160EDBCFE6FF150EF9
:10314000DBCFE6FF040EDBCFE6FF050EDB50E552DA
:10315000E75CE552D880E754E552D880E7545FD960
:10316000030EDB50010B0BE1080EDB5008E0B2D878
:1031700001E08DD0080EDB50BED8080EDB6A170EBA
:10318000DB5007E088D9170EF1D903E1011C01E1FA
:103190007ED0160EDB5016E07ED9300EE66E9FD83C
:1031A00002E1011C74E077D9DFCFE6FF3AEC37F09B
:1031B000E552E552E552F4CF01F00001F31C02E1C3
:1031C000011C65E0050EDBCF00F0160EDB50D88049
:1031D000005409E2050EDBCFE7FF160EDB50E75E79
:1031E000050EE7CFDBFF300EE66E050ECBD94FE1C3
:1031F000390EDB2ADBCFE9FF3A0E01E3DB2ADBCF16
:10320000EAFF090EEFCFDBFFDB500EE044D9090ED9
:10321000ADD902E1011C3BE0390EDB2ADBCFE9FF2F
:103220003A0EEDE3DB2AEBD755D831E1160EDBCFB2
:10323000E6FF080EC3D8E552E7245DD82ED0070E6E
:10324000DB50030A1CE0010A14E0030A07E07BD903
:10325000DBCFEEFF020EDBCFEDFF1FD0F5D8056A06
:1032600003AE02D0046805682CD8BCD805C0EEFFB8
:1032700014D0EAD803BE046824D8B4D80ED063D9D9
:10328000DBCFEFFF0AD07BD905E1011C03E1F36836
:10329000F46810D0FCD801E3DB2A79D9ECEF14F004
:1032A000010EDBCF00F0020EDBCF01F000C0F3FF18
:1032B00001C0F4FF3B0EE15C02E2E16AE552E16E1F
:1032C000CBD029D9020E52EF1AF061D90800F5507F
:1032D000DF6E1200200EE66E080EC2EF1AF03AEC16
:1032E00037F0E552E552E552F3CF00F0F4CF01F0AC
:1032F0000001F31C1200006E016AD950010F4DD974
:103300000050EE260150ED221200045E000E055A18
:10331000F70E04C0DBFFF80E05C0DBFF04C0E9FFB9
:1033200005C0EAFF1200DBCFF4FFF350F45C12009B
:10333000DB50E76E040EE7CFDBFF12000A0EDBCF97
:1033400000F00B0EDBCF01F00C0EDBCF02F00D0E08
:10335000DBCF03F000500110021003101200130E17
:10336000EECFDBFF140EEDCFDBFF130EDBCF00F053
:10337000140EDBCF01F00001800E01141200F70ED5
:10338000DBCF04F0F80EDBCF05F01200050EDB50AA
:10339000E66ED950130F01D9E552E750EE6EED6A93
:1033A00012000A0EDBCF2CF00B0EDBCF2DF00C0E33
:1033B000DBCF2EF00D0EDBCF2FF01200DBCFE6FFC0
:1033C000150EDBCFE6FF050EDB50E552E724E55294
:1033D000E7241200DB50CED8010EF36E060EF3CFB9
:1033E000DBFF1200EE50EFCFEAFFE96E02C0EEFF06
:1033F00003C0EEFF04C0EEFF1200D9CFE6FFDACF24
:10340000E6FFE1CFD9FFE2CFDAFF1200DFCFE6FF20
:10341000E66A66EC38F0E552E552F3501200E76ECA
:10342000080EE7CFDBFF1200EECF00F0EECF01F089
:10343000EFCF02F0036A1200050EDBCF00F0150E8D
:10344000DB50D88000541200010EDBCF02F0020ED8
:10345000DBCF03F0046A1200E552E5CFDAFFE7CFD5
:10346000D9FF12000A0E00C0DBFF0B0E01C0DBFF0C
:103470001200D9500A0FCDEF1AF0F36E070EF3CFFA
:10348000DBFF1200EECF00F0EFCF01F01200010ED3
:10349000DB2A020E1200FC0EDBCFE6FFFD0EDBCFB7
:1034A000E6FF1200005E000E015AF70E00C0DBFFBF
:1034B000F80E01C0DBFF00C0E9FF01C0EAFF120007
:1034C000DA20EA6EEF2AEECFF6FF000EEF22EECF03
:1034D000F7FFEF22EECFF8FF1200040EDBCFE6FF7E
:1034E000130EDB50E552E75C9ADFDB5004DF060E7B
:1034F000DB501200090EDB500A0DF350DF24D00F11
:10350000E76E090EE7CFDBFF65EF19F0DB50F36ED6
:10351000050E93EF19F0F70EDBCF00F0F80EDBCFBE
:1035200001F01200DFCFE6FF6FEF19F028DF030E86
:10353000ECDE14EF1AF0C1EC14F0E552E552E5525E
:10354000E55200091200BDDEEE50EFCFEAFFE96E52
:10355000010E1200130EDB50F36E040E93EF19F000
:10356000040EDB50F36E090E93EF19F0DBCFE6FF8C
:103570006FEF19F0E76E050EE7CFDBFF12008BDF70
:1035800092EF1AF0DBCFE6FF86DF9BEF1AF0D950FF
:10359000F90FE96EFF0E60EF1AF0E96E000EDA2007
:0435A000EA6E1200BD
:0C35A400D9CFE6FFE1CFD9FF180EE126D9
:1035B000110EDB6A120EDB6AFE0EDB50050801E11C
:1035C00077D1FE0EDB50060801E172D1FE0EDB5012
:1035D000070801E16DD1FE0EDB50180801E168D14A
:1035E000FE0EDB50190801E163D1FE0EDB501A0814
:1035F00001E15ED1FE0EDB502F0801E259D1FD0E34
:10360000DB50010801E254D1F90EDBCF00F0FA0ED5
:10361000DBCF01F0FB0EDBCF02F0FC0EDBCF03F0C3
:1036200041EC20F0346E3F0E356E00C02DF001C02D
:103630002EF002C02FF003C030F04AEC20F001E180
:1036400002D1F90EDBCF04F0FA0EDBCF05F0FB0E52
:10365000DBCF06F0FC0EDBCF07F041EC20F0190EBB
:10366000346E400E356E04C02DF005C02EF006C03D
:103670002FF007C030F04AEC20F001E1E4D0F90E61
:10368000DBCF08F0FA0EDBCF09F0FB0EDBCF0AF040
:10369000FC0EDBCF0BF041EC20F0346E400E356EAB
:1036A00008C02DF009C02EF00AC02FF00BC030F07A
:1036B0004AEC20F001E1C7D0F90EDBCF0CF0FA0E96
:1036C000DBCF0DF0FB0EDBCF0EF0FC0EDBCF0FF0EF
:1036D00041EC20F0190E346E410E356E0CC02DF009
:1036E0000DC02EF00EC02FF00FC030F04AEC20F0CD
:1036F00001E1A9D0F90EDBCF10F0FA0EDBCF11F00B
:10370000FB0EDBCF12F0FC0EDBCF13F041EC20F010
:10371000346E410E356E10C02DF011C02EF012C067
:103720002FF013C030F04AEC20F001E18CD0F90EFC
:10373000DBCF14F0FA0EDBCF15F0FB0EDBCF16F06B
:10374000FC0EDBCF17F041EC20F0190E68EC20F0F6
:1037500014C02DF015C02EF016C02FF017C030F099
:103760004AEC20F070E0F90EDBCF18F0FA0EDBCF58
:1037700019F0FB0EDBCF1AF0FC0EDBCF1BF0660E50
:10378000326E336E68EC20F018C02DF019C02EF0A8
:103790001AC02FF01BC030F04AEC20F054E0F90EB4
:1037A000DBCF1CF0FA0EDBCF1DF0FB0EDBCF1EF0E3
:1037B000FC0EDBCF1FF041EC20F068EC20F01CC0C9
:1037C0002DF01DC02EF01EC02FF01FC030F04AECAF
:1037D00020F039E0F90EDBCF20F0FA0EDBCF21F03C
:1037E000FB0EDBCF22F0FC0EDBCF23F0326A336A14
:1037F000C00E68EC20F020C02DF021C02EF022C0B9
:103800002FF023C030F04AEC20F01DE0F90EDBCFA2
:1038100024F0FA0EDBCF25F0FB0EDBCF26F0FC0EFA
:10382000DBCF27F0660E326E336EE60E68EC20F0CA
:1038300024C02DF025C02EF026C02FF027C030F078
:103840004AEC20F035E1F80EDB50070804E0F80EF2
:10385000DB5008082DE1F70EDB50020829E3F20ED9
:10386000DB5026E0F10EDB5023E0F10EDB500508C3
:103870001FE0F10EDB5006081BE0F10EDB500708DD
:1038800017E0F10EDB50180813E0F10EDB501908B9
:103890000FE0F10EDB501A080BE0F10EDB502F08A1
:1038A00007E3FE0EDB50F36EF10EDB50F35C02E13A
:1038B000000E97D32D6A2E6A200E2F6E410E306EA9
:1038C000F90EDBCF32F0FA0EDBCF33F0FB0EDBCF9D
:1038D00034F0FC0EDBCF35F01FEC26F0B3EC26F015
:1038E0002EC0DEFF2FC0DDFF020EDB6A030EDB6A97
:1038F000040EDB6A050EDB6A010EF36E060EF3CFD3
:10390000DBFF070EDB6AF20EDB0498DBEF68FD0ECF
:10391000DB5007E1060EDB6A010EF36E070EF3CFF4
:10392000DBFFFE0EDB5002E0070E8EDBF10EDB50FC
:103930002F0A01E15BD1010A01E152D1030A01E141
:1039400049D1010A01E142D1070A01E139D1010A55
:1039500001E130D1030A01E127D1010A01E11ED1C1
:103960000F0A01E115D1010A01E10CD1030A01E1BD
:1039700003D1010A01E1FAD0070A01E1F1D0010AFD
:1039800001E1E8D0030A01E1DFD0010A01E1D6D06C
:103990003F0A01E1CDD0010A01E1C4D0030A01E1EF
:1039A000BBD0010A01E1B2D0070A01E1A9D0020AA5
:1039B00001E1A0D0010A01E197D00F0A01E18BD00B
:1039C000010A01E182D0030A01E179D0010A6FE026
:1039D000070A68E0010A61E0030A5AE0010A53E0BD
:1039E0001F0A4CE0010A46E0030A40E0010A39E000
:1039F000070A32E0010A2CE0030A25E0010A1DE073
:103A00000C0A15E0070A0DE0010A07E0030A01E0CD
:103A1000F6D03CDB020E88DBE0D038DB010E84DB25
:103A2000E2D0F00EB714B76E010E92DBDCD07F0E41
:103A30006B146B6E020E8CDBD0D0DF0EC614C66E1C
:103A4000800E5EDBA8D00F0EC16E400E59DBA9D0F0
:103A500035DB200E55DBABD00F0EC16E100E50DBE8
:103A6000ACD00F0EC16E080E4BDBADD027DB040EC1
:103A700047DBBFD023DB020E43DBAFD00F0EC16E9E
:103A8000010E3EDBB0D00F0EC16E080E48DB9BD09E
:103A90000F0EC16E040E43DBACD00F0EC16E020ED2
:103AA0003EDB9BD00F0EC16E010E39DB9CD00F0E9A
:103AB000C16EEF0ED214D26E200E31DB78D0DF0E45
:103AC000D514D56E100E2BDB78D0F70ECD14CD6E3D
:103AD000020E1BDB82D0F50ECD14CD6EFD0EB1149F
:103AE000B16E010E12DB7FD07F0EAB14AB6E400EB9
:103AF0000CDB57D07F0EAB14AB6E800E06DB4BD0C9
:103B0000F00EBD14BD6E040E00DB73D0DF0EC614C4
:103B1000C66E080EFADA57D0DF0EC614C66E100E47
:103B2000F4DA4BD0DF0EC614C66E200EEEDA3FD0AC
:103B3000F70EF214F26E800EEDDA2DD0F70EF214BD
:103B4000F26E400EE7DA2DD0F70EF214F26E200E70
:103B5000E1DA2DD0F70EF214F26E100EDBDA2DD072
:103B6000DF0EF014F06E080ED5DA2DD0EF0EF01443
:103B7000F06E040ECFDA3DD0F70EF014F06E020EA8
:103B8000C9DA2BD0EF0EF214F26E010EC3DA2BD08D
:103B90007DDA800EAEDAED6E800E2DD077DA400E33
:103BA000A8DAED6E400E27D071DA200EA2DAED6EA3
:103BB000200E21D06BDA100E9CDAED6E100E1BD0A9
:103BC00065DA080E96DAED6E080E15D05FDA040E8F
:103BD00090DA0FD05BDA020E8CDAED6E020E0BD0AB
:103BE00055DA010E86DAED6E010E05D04FDA040EBD
:103BF0009BDAED6E040EF36E150EF3CFDBFF000EB5
:103C0000DFCF2EF0010EDBCF2FF0800E2E1802E159
:103C1000040E2F1868E0C00E2E1802E1030E2F18B4
:103C20005EE02E5002E1030E2F1855E0400E2E18D4
:103C300002E1020E2F184BE0800E2E1802E1010E59
:103C40002F1841E0C00E2E1801E12F5038E0600E11
:103C50002E1801E12F502FE0300E2E1801E12F50C9
:103C600022E0180E2E1801E12F5010E00C0E2E1835
:103C700041E12F503FE1D20EF1D9340E24DA040E87
:103C8000F36E110EF3CFDBFF030E0AD0650EE6D9FB
:103C9000980E19DA020EF36E110EF3CFDBFF010E50
:103CA000F36E120E25D02F0ED9D9CA0E0CDA010EE2
:103CB000F36E110E1DD0950ED1D9620E17D0470E9E
:103CC000CDD92E0E13D0200EC9D9140E0FD0130E3D
:103CD000C5D90B0E0BD00C0EC1D9070E07D0080E9C
:103CE000BDD9040E03D0060EB9D9020EF36E100E24
:103CF000F3CFDBFFC2D902E0BAEC37F0080EDB6A83
:103D0000090EDB6AFE0EDB5002E0060E9DD9E4D9F7
:103D100001E03BD1A8D939DA110E21DA04E286D9C3
:103D2000FAE3DB2AF8D70F0E6ED905E0010EF36E29
:103D3000080EF3CFDBFF97D96DD904E277D9FCE306
:103D4000DB2AFAD702DA04E0080EDB50020990D928
:103D50008AD960D904E26AD9FCE3DB2AFAD7F5D91B
:103D600004E0080EDB50040983D97DD953D904E25D
:103D70005DD9FCE3DB2AFAD7E8D904E0080EDB5072
:103D8000080976D970D946D904E250D9FCE3DB2A78
:103D9000FAD7DBD904E0080EDB50100969D963D9E2
:103DA00039D904E243D9FCE3DB2AFAD7CED904E0BF
:103DB000080EDB5020095CD956D92CD904E236D93B
:103DC000FCE3DB2AFAD7C1D904E0080EDB50400936
:103DD0004FD9F80EDB50080803E0F70EDB500DE07A
:103DE00042D918D904E222D9FCE3DB2AFAD7ADD9AB
:103DF00004E0080EDB5080093BD9F80EDB500808C0
:103E000011E1F70EDB500EE02ED904D904E20ED9F1
:103E1000FCE3DB2AFAD799D905E0010EF36E090E0F
:103E2000F3CFDBFF59D9FEE0FE0EDB5002E0070EB8
:103E30000BD90E0EDB6AF70EDB505EE0F80EDB509E
:103E400007080DE1080EDB44010BE76E0A0EE7CF11
:103E5000DBFF080EDB507F0BE76E080E04D0090E67
:103E6000DB50E76E0A0EE7CFDBFF0D0EDB6A0C0EB0
:103E7000DB6AF80EDB50F36E0C0EDBCFF4FFF35071
:103E8000F45C1CE2D9500C0FE96EDACFEAFF080EA1
:103E9000DB50EFCFE7FFE75204E0E8427F0BE70695
:103EA000FCE1010B006E0D0EDBCFE7FF0050E726B3
:103EB0000D0EE7CFDBFF0C0EDB2ADBD70D0EDBCFC1
:103EC000E7FF0A0EDB50E7260D0EE7CFDBFFF70E0C
:103ED000DB0404E10D0EDB50010B08E1F70EDB50B3
:103EE000020812E10D0EDB50010B0EE1010EF36E24
:103EF0000E0EF3CFDBFF08D0F80EDB50070804E10D
:103F0000080EDB507F0BB4D80E0EDB5030E186D8A4
:103F1000EF5004E0D950EF0F3FD90BE1040EDB5016
:103F20008DD8080EDBCFEFFF040EDB2AD5D816E1C3
:103F3000E5D61DD906E172D8EF5003E0050EDB2A65
:103F40000DD0050EDB50000809E268D8EF5006E0FE
:103F50000ED904E0050EDB6A040EDB6AF20EDB50BC
:103F6000F36E040EDB50F35C08E1010E3AD0040E50
:103F7000DB5001E0E0D8020E34D07FD806E0020E1C
:103F8000DB6A030EDB6ABAEC37F0A6D801E1B6D6DD
:103F900074D801E1B3D6C1EC37F0000901E1AED627
:103FA000020EDB2A030E01E3DB2A020EDBCF00F058
:103FB000030EDBCF01F0F50EDB5000180FE1F60E1B
:103FC000DB5001180BE1040EDB5001E0B4D8FE0E0B
:103FD000DB5002E0070E38D8030E03D0BAEC37F0FE
:103FE0008DD6006E180EE15C02E2E16AE552E16EE8
:103FF0000050E552E7CFD9FF1200D950130FE96EF8
:10400000DACFEAFF1200DBCFE6FF94EC38F0E5529E
:104010006CEF20F0BAD8120EAFEF20F0050EDB5097
:10402000E76EEF0EDBCFE9FFF00EA8D0E66894EC68
:1040300038F0E552160EDB2A170E1200E76EF30E6B
:10404000DBCFE9FFF40E9AD0DBCFE6FFFE0EDBCF2D
:10405000E6FF21EC28F0E552E5521200F36E0F0E58
:10406000F3CFDBFF1200160EDB6A170EDB6A1200BD
:10407000E76E080EE7CFDBFF1200D950F50FCCEF4B
:1040800020F09A0E326E990E336E1200EF0EB014BD
:10409000B06E1200E2EC26F0010A1200850EEE6E00
:1040A0000F0E1200820EEE6E0F0E1200810EEE6EDB
:1040B0000F0E1200800EEE6E0F0E1200070EB46E81
:1040C0000F0EC16E1200F36E100EF3CFDBFF120065
:1040D000346E420E356E1200150EDBCFE6FF130E66
:1040E000DBCFE9FF140EDBCFEAFFEF50E552E71418
:1040F00012009510956E81DF830EEE6E0F0E12008A
:104100009710976E7ADF4EEF20F09410946E75DF63
:1041100052EF20F09310936E70DF56EF20F0921064
:10412000926E6BDF5AEF20F09610966E66DF840E6B
:10413000EE6E0F0E1200040EDB04E66EF20EDB04D0
:104140007DDFE552E750EF6E1200100E03EF20F016
:104150009810986E52DF860EEE6E0F0E1200DB5036
:10416000026E036AE850005C03500158120056DFEB
:10417000EFCF00F0080EDB50005C1200DBCFEAFF4F
:10418000E750E926000EEA221200160EDBCF00F0FF
:10419000170EDBCF01F01200E96EFF0EDA20EA6E97
:0641A000EE50ED101200CC
:0A41A600D9CFE6FFE1CFD9FF060EE6
:1041B000E126FE0EDB5001E1B9D2FE0EDB50120803
:1041C00001E2B4D2FA0EDBCFE9FFFB0EDBCFEAFF50
:1041D000020EEFCFDBFF010E34DB030EEFCFDBFF70
:1041E000020E2FDB040EEFCFDBFF030E2ADB050EE2
:1041F000EFCFDBFF040EDB5001E198D2040EDB5061
:10420000050801E193D2040EDB50060801E18ED2CD
:10421000040EDB50070801E189D2040EDB501808B8
:1042200001E184D2040EDB50190801E17FD2040EB3
:10423000DB501A0801E17AD2040EDB502F0801E2AC
:1042400075D2020EDB5001E171D2020EDB5005087F
:1042500001E16CD2020EDB50060801E167D2020ECA
:10426000DB50070801E162D2020EDB50180801E1C1
:104270005DD2020EDB50190801E158D2020EDB506C
:104280001A0801E153D2020EDB502F0801E24ED290
:10429000FE0EDB50120A01E12DD2030A01E10AD21F
:1042A000010A01E1F5D11F0A01E1D7D1010A01E1BB
:1042B000C1D1030A01E1A1D1010A01E14FD1070AED
:1042C00001E124D1010A01E114D1030A01E1E6D0A0
:1042D000010A01E1C9D00F0A01E191D0010A5BE0B6
:1042E000030A33E0010A2AE0070A15E0010A0CE09C
:1042F000030A01E01DD2040EE66EE66AC60E006EE9
:104300006A0E64DA040EF3D102DB050EE66ECB0E04
:10431000E66E6A0EEDD1AFDA01E208D2DCDA0C0EFD
:10432000DF5C07E2DF50F76AD10FF66E6A0EB1DA92
:10433000F6D77EC08EF0EBDA0C0ED9D1E8DA0C0E8F
:10434000E66EDE0EE66E6A0ED3D10A0EE66EE66A01
:10435000EB0E006E6A0E3ADA0A0EF9DA1E0EA0DAD9
:10436000100EDF6E010EDB6A29DA02E2FAD9FCD701
:104370004ADB140EDF6E010EDB6A20DA02E2F1D9AD
:10438000FCD7CFDA180EDF6E010EDB6A17DA01E315
:10439000E0D0E7D9FBD76FDA01E2C8D19CDA120E80
:1043A000DF5C07E2DF50F76AF60FF66E6A0E71DA2D
:1043B000F6D77EC08EF0020E17DB010EDB50DF5CFD
:1043C00004E222DA0C0EBDDAF8D7DF504BDA010E28
:1043D000DB500D0FBCDA0EDB01E1A8D1C8DAE2DA5E
:1043E000EDD902E2BED9FCD7AFDAE8D902E2B9D9F9
:1043F000FCD706DBE3D901E3ACD0B3D9FBD7DF6A46
:104400001C0EDF5C07E2DF50F76A090FF66E6B0ED9
:1044100040DAF6D7F3D966DA040EDF5C04E2F4D9A9
:10442000090E8FDAF9D7020EBADA040EDF5C04E265
:10443000EBD90D0E86DAF9D7040EB1DA040EDF5C83
:1044400004E2E2D9110E7DDAF9D7060ECDDA010EBB
:10445000DB50DF5C04E2D8D9160E73DAF8D7DF50F0
:1044600064DA0D0EEF6E40D052DA040EE66E260EC0
:10447000E66E6B0E8ED9BEDA01E158D178DA92DAA7
:104480009DD902E26ED9FCD75FDA98D902E269D9E8
:10449000FCD7B6DA93D95DE264D9FCD7DF6A100E97
:1044A000DF5C07E2DF50F76A2B0FF66E6B0EF1D977
:1044B000F6D7A4D917DA040EDF5C04E2A5D9030EFF
:1044C00040DAF9D7020E6BDA040EDF5C04E29CD905
:1044D000070E37DAF9D7040E62DA040EDF5C04E265
:1044E00093D90B0E2EDAF9D712DA010EDB50170F23
:1044F000FED0040EE66EE66A3C0E006E6B0E66D9C8
:10450000040EE66E3C0EE66E6B0EF2D000DA0B0E79
:10451000E66E410EE66E6B0E3CD9100EC1D9020E4E
:10452000DF6E010EDB6A4AD902E21BD9FCD76BDAD7
:10453000060EDF6E010EDB6A41D902E212D9FCD70A
:10454000F0D90A0EDF6E010EDB6A38D902E209D912
:10455000FCD7CED9F4CF01F0040E4DD0D8D90C0E33
:10456000E66E4D0EE66E6B0E14D90A0E99D9DF6A0F
:10457000A9D9DF2A7CD90A0E0001A15DF9E1DF503B
:10458000DAD9EF6ADF6A0C0EDF5C07E2DF50F76A08
:104590004D0FF66E6B0E7DD9F6D70001310E8E6F82
:1045A000B6D90C0ED4D90A0E7BD9DF6A040EDF5CB3
:1045B00008E288D95CD92C0E0001A15D02E1DF2A56
:1045C000F5D74AD9F3CF00F0F4CF01F02FD9CFD9E6
:1045D000020E66D9DF6A050EDF5C08E273D947D99F
:1045E0000A0E0001A15D02E1DF2AF5D7DF0634D90A
:1045F000F4CF01F0020EF7D897D0DF6A1C0EDF5C13
:1046000007E2DF50F76A5A0FF66E6B0E42D9F6D703
:10461000DF6A100EDF5C07E200D905E0FED8E66E27
:104620000A0E8FD9F6D70A0E2FD90B0EDF241AD90E
:104630000C0E5CD00DD901E279D04DD90A0EDF5CA9
:1046400007E2DF50F76A770FF66E6B0E22D9F6D7C6
:104650007EC08CF05CD90A0E4AD0FAD867E33BD909
:104660000D0EDF5C07E2DF50F76A820FF66E6B0E0D
:1046700010D9F6D77EC08DF0020E98D9010E72D9EE
:1046800055E3020E48D97EC08FF041D90D0E2FD0D0
:10469000DFD84CE320D90B0EDF5C07E2DF50F76A6E
:1046A000900FF66E6B0EF5D8F6D77EC08DF02FD931
:1046B0000B0E1DD0DF6A1D0EDF5C07E2DF50F76ACC
:1046C0009C0FF66E6B0EE5D8F6D7DF6A100EDF5C36
:1046D00007E2A3D805E0A1D8E66E0B0E32D9F6D7D3
:1046E0000B0ED2D80C0EDF24BDD80D0EDF24C7D898
:1046F000DAD81AD0030EE66EE66ABA0E006E6B0EBA
:1047000065D8030E24D9060ECBD80001666BF00ED7
:10471000E66E000E7BD9E66E68EC34F0E552E552A9
:10472000E552E552000902E1010E03D0000E01D06E
:10473000000E006E060EE15C02E2E16AE552E16EF7
:104740000050E552E7CFD9FF120037D91ED9050E28
:10475000DBCFE6FFD2EC1AF0006E100EE15E0050E7
:104760001200DF50E8D8EF50E66E2FD9E552E7503F
:10477000EF6EDF2A010EDB2A1200ECD87E0EE66E09
:10478000000EE66E40EC36F0036E070EE15E03505D
:10479000120089D8B7EF24F0ABD8F3CF00F0F4CFF4
:1047A00001F01200C2D8E552E750EF6EDF2A120086
:1047B000FDD8EECFE6FFEFCFE6FF1200040EF36E5A
:1047C000010EDBCFF4FFF350F45C1200C3D8840E6B
:1047D000E66E000EE66E2BEC34F0036E070EE15E23
:1047E000035087EF24F0E76EF80EDBCFE9FFF90EF8
:1047F00087D8F3CFEEFF01C0EDFF1200BFD8EECF98
:10480000E6FFEFCFE6FF1200DF50EA6A7E0FE96EA7
:10481000000EEA22EF50E66E1200DF50E76EF60E51
:10482000DBCFE9FFF70E6CD8EF501200F80EDBCFAC
:10483000E9FFF90EDBCFEAFFF3CFEEFF01C0EDFF9A
:104840001200E76EFA0EDBCFE9FFFB0E80EF24F0DB
:1048500095D8010EB2EF24F0DF506DD8EF6A0A0E42
:10486000D5D8BBD062D80D0EEF6E87EF24F063D899
:10487000A1C0EFFF120082D8030EB2EF24F0E66E63
:10488000840EE66E000E1200DF244FD8220EEF6E6B
:104890001200F7220800F550E66EDF50D2EF23F049
:1048A000B5D8A5EF23F089D8000EE66EE66A6DD87C
:1048B000030EDBCFE6FF22EC04F0006E100EE15E8B
:1048C0000050120054D8010EE66EA10EE66E000EE6
:1048D0003CDFDF50120092DF750E006E710E4DDF6F
:1048E000DF6A1200700E006E710E47DFDF6A120081
:1048F0006CD8EF6A100EE66EF00EE66E000E6DD00C
:10490000DBCFEAFFE750E926000EEA221200020E92
:10491000DBCFE6FF12004CDF750E006E710EBDEFAF
:1049200023F03ADF020EF3EF23F0EA6A840FE96E18
:10493000000EEA221200EA6A600FE96E000EEA2217
:104940001200DF24D2EF23F05ED80B0E64D097DF85
:10495000C9EF23F0016E026A00C0E6FFE66E02C0F6
:10496000E6FF1200D880EE54000EED541200000E47
:10497000E66EE66A040EDBCFE6FF1200FC0EDBCF2C
:10498000E9FFFD0EDBCFEAFF12009A0EE66E990EEC
:10499000E66E190EE66E410EE66EE66A120008DF5C
:1049A00072EF24F0150E7CDF070E35D0E76EFC0E9B
:1049B000DBCFE9FFFD0E80EF24F0E66E000EE66E21
:1049C000E66AE66A080EE66E1200010EDB50EA6A3D
:1049D000F00FE96E000EEA221200E66E42EC33F0B0
:1049E000E552E552E552120096DF010EF3CFDBFFF0
:1049F000DF6A1200090E54DF450E0001685D1200E7
:104A000090DF0F0E08D0C8DE16EF24F0E66E600EC1
:0E4A1000E66E000E1200DF6E010EDB6A120071
:024A1E00379EC1
:104A200005D0379E2FAE02D02F6C378E2FC029F0C5
:104A3000286A3B6A3A6A860E2A6E2B6A6CEF27F068
:104A4000379E08D0379E2FAE05D02E6C2F1EE86AF9
:104A50002F22378E2FC029F02EC028F03B6A3A6AE9
:104A60008E0E2A6E2B6A6CEF27F0357E376AA8EC23
:104A700027F0C0EC27F037B650EF27F037A20AD066
:104A800037AA03D037BE50EF27F037A45CEF27F0EA
:104A900059EF27F037AA05D037AC5CEF27F059EF74
:104AA00027F037A00AD037A808D037BE04D037A4E3
:104AB00002D065EF27F069EF27F03A6A2B6A35508C
:104AC000305C396E10E32DC03BF02EC028F02FC0B3
:104AD00029F030C038F032C02DF033C02EF034C091
:104AE0002FF0373A09D032C03BF033C028F034C041
:104AF00029F035C038F0396C379E37BC378E38C056
:104B00002AF037B098EF27F01A0E396098EF27F0A7
:104B10002A6A306A37A408D02D6C2E1E2F1E301E34
:104B2000E86A2E222F22302237AC08D03B6C281E98
:104B3000291E2A1EE86A282229222A222C6A395292
:104B400007E030342F322E322D322C32392EF9D765
:104B50002D503B262E5028222F50292230502A2219
:104B60002CC03AF0379E2AAE0BD03A6C3B1E281E62
:104B7000291E2A1EE86A3B22282229222A22378E51
:104B80002AA006D0D880293228323B323A32382A3D
:104B900038C02AF06CEF27F0376AA8EC27F0C0EC99
:104BA00027F037B650EF27F037A205D037BA50EFCD
:104BB00027F057EF27F037BA63EF27F037A005D07B
:104BC00037B850EF27F063EF27F037B857EF27F0EB
:104BD0002B6A7F0E30242A6EE86A2B2235502A5E1B
:104BE000E86A2B5A1A0E386E306A3A6A3B6A286AAB
:104BF000296A32502D5E33502E5A34502F5A000EEF
:104C0000305A09E732502D2633502E2234502F22AD
:104C1000000E302201D03A8AD8902D362E362F360B
:104C20003036D8903A363B3628362936382EE1D7FA
:104C30002F502E102D10D8A43A8A6CEF27F0376A27
:104C4000A8EC27F0C0EC27F037B650EF27F037A2DA
:104C500005D037B850EF27F057EF27F037AA05D027
:104C600037B050EF27F057EF27F037B002D037A812
:104C700002D063EF27F02B6A355030242A6EE86AA1
:104C80002B227E0E2A5EE86A2B5A3A6A3B6A286A11
:104C9000296A34502F02F4CF29F0F3CF28F0335093
:104CA0002F02F3503B26F4502822000E29223450C4
:104CB0002E02F3503B26F4502822000E29223250B7
:104CC0002F02F3503A26F4503B22000E28222922CC
:104CD00033502E02F3503A26F4503B22000E282285
:104CE000292234502D02F3503A26F4503B22000E74
:104CF0002822292232502E02F4503A26000E3B225E
:104D00002822292233502D02F4503A26000E3B224D
:104D1000282229226CEF27F0376AA8EC27F037B653
:104D200096EF26F037A20AD037B403D07F0E2F6E4D
:104D300019D0800E2F6E16D02F6A14D037B0FCD742
:104D4000870E3060F1D77E0E3064F6D7860E305C69
:104D500004E0D8902F32302AF9D737A403D02F6C33
:104D60002FAEEAD71200376AA8EC27F037B6BDEFAE
:104D700026F037A20ED037B405D07F0E2F6EFF0E6F
:104D80002E6E1FD0800E2F6E2E6A1BD02F6A2E6AB9
:104D900018D037B0FBD78F0E3060EDD77E0E306461
:104DA000F5D78E0E305C05E0D8902F322E32302AA7
:104DB000F8D737A406D02E6C2F1EE86A2F222FAE0C
:104DC000E5D71200FBEC26F037B6000C37B0010C2B
:104DD000000CFBEC26F037B6000C37B0000C37B4F3
:104DE000000C010CFBEC26F037B6000C37B0000CC1
:104DF00037A4000C010C376AA8EC27F0C0EC27F0B0
:104E000037B6120037AE08D037A004D037A802D08A
:104E100037801200379012003550305C0BE134506F
:104E20002F5C08E133502E5C05E132502D5C02E12D
:104E300037801200D8A002D0378E10D0305035C045
:104E400030F0356E2F5034C02FF0346E2E5033C0FA
:104E50002EF0336E2D5032C02DF0326E3550305C56
:104E600010E0FF0F09E0379037B403D037AE378436
:104E7000120037AE37941200352AD89034323332CC
:104E8000323232502D5E33502E5A34502F5A2FBEAC
:104E9000EAD7D8902D362E362F36302EF8D7C8D7F1
:104EA0007F0E306EFF0E2F6E2E6E2D6E12007F0E57
:104EB00037BEFF0E306E02D07F0E306E800E2F6E2A
:104EC0002E6A2D6AF3D737AE04D0800E306E2F6A6B
:104ED000F7D7306A2F6AF4D7295028103B103A10C0
:104EE000F8E02BBEF0D729BE0CD02A502B10EBE0F7
:104EF000D8903A363B36283629362A06D8A02B06D3
:104F0000F2D72B50D4E12A28D2E03AAE11D07F0E4E
:104F10003A1402E13BA00CD03B2AE86A282229225D
:104F200007E3D880293228323B322A2A2A28BFE0D8
:104F30002A50C9E03BC02DF028C02EF029342F6E36
:104F40002A30306E2F32309E37BE308E56EF27F02B
:104F50002F36303602E33784377E06E13780306AF9
:104F60002F6A2E6A2D6A1200302803E0D8802F3273
:104F70001200D8902F3202E13782120037861200D9
:104F80003436353602E3378C377E06E13788356AAA
:104F9000346A336A326A1200352803E0D88034322A
:104FA0001200D8903432EAE1378A12002EC03AF06B
:104FB0002E503302F4CF2DF0F3CF2CF02F503402CB
:104FC000F4CF2FF0F3CF2EF03302F3502D26F45010
:104FD0002E22E86A2F223A503402F3502D26F45044
:104FE0002E22E86A2F22000C2FC03BF02EC03AF090
:104FF0002E503302F4CF2DF0F3CF2CF02F5034028B
:10500000F4CF2FF0F3CF2EF03302F3502D26F450CF
:105010002E22E86A2F223A503402F3502D26F45003
:105020002E22E86A2F2234AE1AEF28F03A502E5E74
:105030003B502F5A3BAE000C33502E5E34502F5A4B
:02504000000C62
:0E504200D9CFE6FFE1CFD9FFE652FD0EDB50DD
:1050500002E1DF6A02D0010EDF6EFE0EDB502F0A86
:1050600001E12FD2010A01E123D2030A01E117D2A3
:10507000010A01E10BD2070A01E1FFD1010A01E1B6
:10508000F3D1030A01E1E7D1010A01E1DBD10F0A03
:1050900001E1CFD1010A01E1C1D1030A01E1B3D19C
:1050A000010A01E1A5D1070A01E197D1010A01E155
:1050B00089D1030A01E17BD1010A01E16DD13F0AE7
:1050C00001E15FD1010A01E151D1030A01E143D1BC
:1050D000010A01E135D1070A01E127D1020A01E104
:1050E00019D1010A01E10BD10F0A01E1FAD0010A3D
:1050F00001E1ECD0030A01E1DED0010A01E1CED0EA
:10510000070A01E1C1D0010A01E1B4D0030A01E1BB
:10511000A7D0010A01E19AD01F0A01E18DD0010A4E
:1051200001E181D0030A01E175D0010A69E0070AB3
:105130005DE0010A52E0030A46E0010A39E00C0A88
:105140002AE0070A1BE0010A0EE0030A01E0C4D1CD
:10515000C9D9FD0E9614966EDF50E8B08D82E8B086
:10516000B9D18D92B7D1BED9FE0E9614966EDF508E
:10517000E8B08D80E8B0AED18D90ACD1F00EB71410
:10518000B76EFE0E9814986EDF50E8B08F80E8B0CE
:10519000A1D18F909FD17F0E6B146B6EFD0E981472
:1051A000986EDF50E8B08F82E8B094D18F9292D1A0
:1051B000DF0EC614C66E7F0E99D9E8B08E8EE8B0A9
:1051C00089D18E9E87D10F0EC16EBF0E8FD9E8B0E8
:1051D0008E8CE8B07FD18E9C7DD19CD9DF0E86D994
:1051E000E8B08E8AE8B076D18E9A74D10F0EC16E77
:1051F000EF0E7CD9E8B08E88E8B06CD18E986AD179
:105200000F0EC16EF70E72D9E8B08E86E8B062D18B
:105210008E9660D17FD9FB0E69D9E8B08E84E8B054
:1052200059D18E9457D176D9FD0E60D9E8B08E82CF
:10523000E8B050D18E924ED10F0EC16EFE0E56D9EF
:10524000E8B08E80E8B046D18E9044D10F0EC16E8A
:10525000F70E5CD9E8B08986E8B03CD189963AD19E
:105260000F0EC16EFB0E52D9E8B08984E8B032D17E
:10527000899430D10F0EC16EFD0E48D9E8B08982F5
:10528000E8B028D1899226D10F0EC16EFE0E3ED90C
:10529000E8B08980E8B01ED189901CD10F0EC16E94
:1052A000EF0ED214D26EDF0E31D9E8B0898AE8B0A1
:1052B00011D1899A0FD1DF0ED514D56EEF0E26D9F4
:1052C000E8B08988E8B006D1899804D1F70ECD14EA
:1052D000CD6EFD0E0FD9E8B08B82E8B0FBD08B927B
:1052E000F9D0F50ECD14CD6EFD0EB114B16EFE0EDB
:1052F00001D9E8B08B80E8B0EDD08B90EBD07F0E79
:10530000AB14AB6EBF0EF6D8E8B08B8CE8B0E2D031
:105310008B9CE0D07F0EAB14AB6E7F0EEBD8E8B069
:105320008B8EE8B0D7D08B9ED5D0F00EBD14BD6E5D
:10533000FB0EE0D8E8B08B84E8B0CCD08B94CAD018
:10534000DF0EC614C66EF70ED5D8E8B08B86E8B06F
:10535000C1D08B96BFD0DF0EC614C66EEF0ECAD872
:10536000E8B08B88E8B0B6D08B98B4D0DF0EC61406
:10537000C66EDF0EBFD8E8B08B8AE8B0ABD08B9A90
:10538000A9D0F70EF214F26E7F0EB8D8E8B08A8E6C
:10539000E8B0A0D08A9E9ED0F70EF214F26EBF0E37
:1053A000ADD8E8B08A8CE8B095D08A9C93D0F70E3F
:1053B000F214F26EDF0EA2D8E8B08A8AE8B08AD082
:1053C0008A9A88D0F70EF214F26EEF0E97D8E8B0F2
:1053D0008A88E8B07FD08A987DD0DF0EF014F06E16
:1053E000F70E8CD8E8B08A86E8B074D08A9672D06E
:1053F000EF0EF014F06EFB0E81D8E8B08A84E8B0AE
:1054000069D08A9467D0F70EF014F06EFD0E76D84E
:10541000E8B08A82E8B05ED08A925CD0EF0EF214D7
:10542000F26EFE0E6BD8E8B08A80E8B053D08A9056
:1054300051D058D87F0E66D8E8B08C8EE8B04AD0EC
:105440008C9E48D04FD8BF0E5DD8E8B08C8CE8B0A9
:1054500041D08C9C3FD046D8DF0E54D8E8B08C8A1F
:10546000E8B038D08C9A36D03DD8EF0E4BD8E8B0A3
:105470008C88E8B02FD08C982DD034D8F70E42D835
:10548000E8B08C86E8B026D08C9624D02BD8FB0EC2
:1054900039D8E8B08C84E8B01DD08C941BD022D8C9
:1054A000FD0E30D8E8B08C82E8B014D08C9212D0C7
:1054B00019D8FE0E27D8E8B08C80E8B00BD08C90BD
:1054C00009D010D8FB0E9614966EDF50E8B08D848C
:1054D000E8A08D94010E01D0000EE552E552E7CF11
:1054E000D9FF1200EF0EB014B06E12009714976E31
:1054F000DF5012009414946EDF5012009314936ED8
:10550000DF5012009514956EDF5012009214926EC7
:0E551000DF501200070EB46E0F0EC16E1200B7
:02551E00D9CFE3
:10552000E6FFE1CFD9FF100EE126FC0EC214C26ED9
:10553000FD0EDB50010A51E0030A49E0010A41E097
:10554000070A39E0010A31E0030A2AE0010A23E0F0
:105550000F0A1DE0010A16E0030A0FE0010A08E045
:10556000070A01E097D0A4D97F0E8CD9030E3AD058
:105570009FD93F0E87D9040E35D09AD91F0E82D9F4
:10558000050E30D095D90F0E7DD9060E2BD090D9AF
:1055900079D9070E27D08CD9030E74D9080E22D0E2
:1055A000B8D9010E6FD9090E1DD0B3D92F0E9210A4
:1055B000926E0A0E17D0ADD90F0E9210926E0B0E8E
:1055C00011D0A7D9070E9210926E0C0E0BD0A1D954
:1055D000030E9210926E0D0E05D09BD9010E921003
:1055E000926E0E0EC16EFC0EDB50030A25E0010A1E
:1055F0000FE0030A06E0010A4DE1CF0EC11472D993
:105600000CD0CF0EC114C16E100EC1106BD916D0C4
:10561000CF0EC114C16E200E3BD9040EDB6A050EFD
:10562000DB6AA00EF36E060EF3CFDBFF400EF36EC7
:10563000070EF3CFDBFF14D0300E2AD9D950F40F68
:10564000E96EFF0EDA20EA6E040EEECFDBFF050EE8
:10565000EECFDBFF060EEECFDBFF070EEECFDBFF5C
:10566000FE0EDB50140A3EE0070A39E0010A34E07E
:10567000030A2FE0010A2AE01F0A25E0010A20E0C0
:10568000030A1BE0010A16E0070A11E0010A0CE018
:10569000030A07E0006A016A800E026EBF0E036E05
:1056A000DFD00AD92C0E20D007D9280E1DD004D95E
:1056B000240E1AD001D9200E17D0FED81C0E14D0FB
:1056C000FBD8180E11D0F8D8140E0ED0F5D80C0E49
:1056D0000BD0F2D8080E08D0EFD8040E05D0C30EB8
:1056E000C21403D0E9D8100EC210C26E860EC06E6E
:1056F000010EC210C26E0F0EE66EE66A93EC37F032
:10570000E552E552020EC210C26EC2B2FED7C450BC
:10571000E66ED950080FEED8030EE76E080EDBCF09
:1057200000F0090EE7500016016A00C001F0006A9F
:10573000E9D8C350E66ED9500A0FDCD8FF0EE76EE9
:105740000A0EDBCF02F00B0EE7500216036A080EBA
:10575000DB500210006E090EDB500310016ED2D830
:10576000080EDBCF2EF0090EDBCF2FF020EC25F05A
:10577000A7D8326A336A800E346E440E356ECCEC94
:1057800025F00C0E2DC0DBFF0D0E2EC0DBFF0E0E24
:105790002FC0DBFF0F0E30C0DBFFBFD8EECF04F011
:1057A000EECF05F0EECF06F0EFCF07F00C0EDBCF1B
:1057B0000CF00D0EDBCF0DF00E0EDBCF0EF00F0E4A
:1057C000DBCF0FF0040EDBCF14F0050EDBCF15F0AE
:1057D000060EDBCF16F0070EDBCF17F09ED8EECF0C
:1057E00018F0EECF19F0EECF1AF0EFCF1BF018C083
:1057F00032F019C033F01AC034F01BC035F014C0B9
:105800002DF015C02EF016C02FF017C030F035EC7B
:1058100025F02DC010F02EC011F02FC012F030C0B6
:1058200013F057D80CC02DF00DC02EF00EC02FF085
:105830000FC030F01FEC26F02DC008F02EC009F08C
:105840002FC00AF030C00BF044D804C02DF005C0C2
:105850002EF006C02FF007C030F036EC25F030D81F
:1058600000C02CF001C02DF002C02EF003C02FF0BC
:10587000100EE15C02E2E16AE552E16EE552E7CF2B
:10588000D9FF12009710976E2F0E9210926E120091
:10589000C110C16E42D8F80EDBCFEEFFF90EDBCFA0
:1058A000EEFFFA0EDBCFEEFFFB0EDBCFEEFF1200BA
:1058B00030D8070EB46E1200C30EC214C26E1200AE
:1058C0002DC000F02EC001F02FC002F030C003F058
:1058D00012002DC032F02EC033F02FC034F030C093
:1058E00035F01200C16EDE6ADE6ADE6ADD6ADD5204
:1058F000DD521200E96EDACFEAFFE552E750EE6EB4
:10590000ED6A1200080E00C0DBFF090E01C0DBFFCC
:105910001200EF0ED214D26E1200D9CFE9FFDACF07
:04592000EAFF120088
:0C592400D9CFE6FFE1CFD9FFFE0EDB502B
:105930002F0A01E1B9D1010A01E1AFD1030A01E166
:10594000A6D1010A01E19DD1070A01E194D1010A22
:1059500001E18BD1030A01E182D1010A01E179D190
:105960000F0A01E170D1010A01E167D1030A01E1E7
:105970005CD1010A01E151D1070A01E146D1010AD6
:1059800001E13BD1030A01E130D1010A01E125D156
:105990003F0A01E11AD1010A01E10ED1030A01E136
:1059A00002D1010A01E1F6D0070A01E1EAD0020AB8
:1059B00001E1DED0010A01E1D2D00F0A01E1C6D037
:1059C000010A01E1BAD0030A01E1AED0010A01E106
:1059D000A0D0070A01E198D0010A01E18DD0030AA5
:1059E00001E182D0010A01E177D01F0A01E16FD005
:1059F000010A66E0030A5DE0010A53E0070A49E094
:105A0000010A40E0030A36E0010A2BE00C0A1EE01E
:105A1000070A14E0010A0CE0030A01E04ED152D952
:105A2000020E9610966E8450020B01E147D143D1CD
:105A300049D9010E9610966E845034D1F00EB714E9
:105A4000B76E010E9810986E86502CD17F0E6B1495
:105A50006B6E020E9810986E8650020B01E12ED1EB
:105A60002AD1DF0EC614C66E800E30D9800B01E13C
:105A700025D121D10F0EC16E400E28D9400B01E176
:105A80001DD119D137D9200E21D9200B01E116D112
:105A900012D10F0EC16E100E19D9100B01E10ED1EB
:105AA0000AD10F0EC16E080E11D9080B01E106D103
:105AB00002D120D9040E0AD9040B01E1FFD0FBD09A
:105AC00019D9020E03D9020B01E1F8D0F4D00F0E60
:105AD000C16E010EFBD8E6D00F0EC16E080E06D9BE
:105AE000080B01E1EBD0E7D00F0EC16E040EFED81B
:105AF000040B01E1E3D0DFD00F0EC16E020EF6D829
:105B0000020B01E1DBD0D7D00F0EC16E010EEED833
:105B1000C9D00F0EC16EEF0ED214D26E200EE6D891
:105B2000200B01E1CBD0C7D0DF0ED514D56E100EFF
:105B3000DDD8100B01E1C2D0BED0F70ECD14CD6E72
:105B4000020EC8D8020B01E1B9D0B5D0F50ECD14C4
:105B5000CD6EFD0EB114B16E010EBCD8A3D07F0E78
:105B6000AB14AB6E400EB6D8400B01E1A7D0A3D06A
:105B70007F0EAB14AB6E800EADD8800B01E19ED0D2
:105B80009AD0F00EBD14BD6E040EA4D8040B01E132
:105B900095D091D0DF0EC614C66E080E9BD8080BA8
:105BA00001E18CD088D0DF0EC614C66E100E92D8DC
:105BB000100B01E183D07FD0DF0EC614C66E200E1D
:105BC00089D8200B01E17AD076D0F70EF214F26E6C
:105BD000800E84D8800B72E06ED0F70EF214F26E55
:105BE000400E7CD8400B6AE066D0F70EF214F26EDD
:105BF000200E74D8200B62E05ED0F70EF214F26E25
:105C0000100E6CD8100B5AE056D0DF0EF014F06E68
:105C1000080E64D8080B52E04ED0EF0EF014F06E70
:105C2000040E5CD8040B4AE046D0F70EF014F06E78
:105C3000020E54D8020B42E03ED0EF0EF214F26E88
:105C4000010E4CD82FD03ED8800E4CD8800B36E0B9
:105C500032D038D8400E46D8400B30E02CD032D865
:105C6000200E40D8200B2AE026D02CD8100E3AD88F
:105C7000100B24E020D026D8080E34D8080B1EE0E4
:105C80001AD020D8040E2ED8040B18E014D01AD83D
:105C9000020E28D8020B12E00ED014D8010E951077
:105CA000956E8350010B0AD00DD8040E9610966E97
:105CB0008450040B03E0010E01D0FF0EE552E7CF44
:105CC000D9FF1200EF0EB014B06E12009710976E4D
:105CD000855012009410946E825012009310936EAF
:105CE000815012009510956E835012009210926EA2
:0E5CF00080501200070EB46E0F0EC16E12002F
:025CFE00D9CFFC
:105D0000E6FFE1CFD9FFE652FE0EDB502F0A01E19C
:105D100011D1010A01E10AD1030A01E102D1010A0C
:105D200001E1FBD0070A01E1F4D0010A01E1EDD065
:105D3000030A01E1E6D0010A01E1DFD00F0A01E127
:105D4000D8D0010A01E1D3D0030A01E1CCD0010A85
:105D500001E1C5D0070A01E1BED0010A01E1B7D0D7
:105D6000030A01E1B0D0010A01E1A9D03F0A01E133
:105D7000A2D0010A01E19BD0030A01E194D0010AFB
:105D800001E18DD0070A01E186D0020A01E17FD04E
:105D9000010A01E178D00F0A01E173D0010A6DE038
:105DA000030A67E0010A61E0070A5DE0010A57E0C3
:105DB000030A51E0010A4BE01F0A47E0010A41E0F3
:105DC000030A3AE0010A33E0070A2CE0010A25E061
:105DD000030A1EE0010A17E00C0A10E0070A0CE0B3
:105DE000010A08E0030A01E0AAD08450020B01E195
:105DF0009FD09AD084509BD0865099D08650020B69
:105E000001E196D091D08550800B01E191D08CD0EA
:105E10008550400B01E18CD087D08550200B01E1EB
:105E200087D082D08550100B01E182D07DD0855083
:105E3000080B01E17DD078D08550040B01E178D0CA
:105E400073D08550020B74E06FD0855070D08050B5
:105E5000080B6EE069D08050040B6AE065D080507A
:105E6000020B66E061D0805062D08050200B60E071
:105E70005BD08050100B5CE057D08250020B58E092
:105E800053D0825054D08250400B52E04DD08250BB
:105E9000800B4EE049D08250040B4AE045D082503E
:105EA000080B46E041D08250100B42E03DD08250BA
:105EB000200B3EE039D08150800B3AE035D0815044
:105EC000400B36E031D08150200B32E02DD0815094
:105ED000100B2EE029D08150080B2AE025D08150EC
:105EE000040B26E021D08150020B22E01DD081500E
:105EF0001ED08350800B1CE017D08350400B18E05D
:105F000013D08350200B14E00FD08350100B10E0FF
:105F10000BD08350080B0CE007D08350040B08E033
:105F200003D08350020B04E0010E02D08350010B1A
:105F3000DF6E05D08450040B01E0010EDF6EDF50F0
:105F400003E1010EE66E01D0E66AFE0EDBCFE6FF4E
:105F500021EC28F0E552E552E552E552E7CFD9FFB2
:025F600012002D
:0E5F6200D9CFE6FFE1CFD9FF090EE126F80EF8
:105F7000DBCF00F0F90EDBCF01F0FA0EDBCF02F041
:105F8000FB0EDBCF03F0326A336A800E346E400EB4
:105F9000356E00C02DF001C02EF002C02FF003C0FE
:105FA00030F0F2EC26F0010A01E1C9D0F80EDBCFA7
:105FB00004F0F90EDBCF05F0FA0EDBCF06F0FB0E96
:105FC000DBCF07F0326AF20E336E5D0E346E480E90
:105FD000356E04C02DF005C02EF006C02FF007C0AE
:105FE00030F0E9EC26F0010A01E1A9D02D6A2E6A11
:105FF000800E2F6E3F0E306EF80EDBCF32F0F90EB2
:10600000DBCF33F0FA0EDBCF34F0FB0EDBCF35F015
:10601000CCEC25F02DC00CF02EC00DF02FC00EF0F2
:1060200030C00FF0326A240E336E740E346E490E97
:10603000356E1FEC26F02DC008F02EC009F02FC0E1
:106040000AF030C00BF0326A336A346A400E356EA3
:10605000CCEC25F02DC004F02EC005F02FC006F0CA
:1060600030C007F0CD0E326ECC0E336E0C0E346E97
:10607000400E356ECCEC25F02DC000F02EC001F0A6
:106080002FC002F030C003F0326A336A346A3F0E28
:10609000356E36EC25F0050E2DC0DBFF060E2EC04A
:1060A000DBFF070E2FC0DBFF080E30C0DBFF050E45
:1060B000DBCF2DF0060EDBCF2EF0070EDBCF2FF05F
:1060C000080EDBCF30F0B3EC26F0020E2EC0DBFF63
:1060D000030E2FC0DBFF040EDB6A3ED830E0DE6A21
:1060E000DD6ABAEC37F0C1EC37F0000906E0DF2AD0
:1060F000010E01E3DB2ABAEC37F0FC0EDB50DF18AF
:1061000007E1FD0EDB50DE52DD1802E1010E18D072
:10611000020EDBCFE6FF030EDBCFE6FF93EC37F09A
:10612000E552E552040EDB5006E1010EF36E040E5B
:10613000F3CFDBFF02D0040EDB6A0ED8D4E1000EF1
:10614000006E090EE15C02E2E16AE552E16E005088
:10615000E552E7CFD9FF1200DBCFE6FFFE0EDBCF23
:0E616000E6FF21EC28F0E552E552000912009E
:02616E00D9CF87
:10617000E6FFE1CFD9FF020EE126FE0EDB501B0841
:1061800004E0FE0EDB50030807E1DAD8FF0ED880EA
:10619000EE54030EED5402E2000EBAD0D1D8EE5008
:1061A000ED1006E1FE0EDB501B0802E1BD6A09D0CE
:1061B000C7D8EE50ED1007E1FE0EDB50030803E1F7
:1061C000B76A010EA5D00C6A0D6A800E0E6E400EE5
:1061D0000F6EFC0EDBCF2EF0FD0EDBCF2FF020EC90
:1061E00025F02DC010F02EC011F02FC012F030C0DD
:1061F00013F0ADD80CC02DF00DC02EF00EC02FF056
:106200000FC030F01FEC26F02DC008F02EC009F0B2
:106210002FC00AF030C00BF0FB0EDBCF18F018C017
:106220002FF00FEC25F02DC014F02EC015F02FC06C
:1062300016F030C017F08BD808C02DF009C02EF032
:106240000AC02FF00BC030F01FEC26F02DC004F078
:106250002EC005F02FC006F030C007F0326AC00E25
:10626000336E7F0E346E440E356ECCEC25F02DC0AF
:1062700000F02EC001F02FC002F030C003F0326AEF
:10628000336A346A3F0E356E36EC25F0B3EC26F0F7
:106290002EC0DEFF2FC0DDFFC00EB16EFE0EDB5044
:1062A0001B081BE1FB0EDB50CB6E3ED8BE6EDECF73
:1062B00002F0DDCF03F0040ED89002360336E80476
:1062C000FBE1CF0EBD140210E850BD6E060ECA10E1
:1062D000CA6E0C0EBD10BD6E1AD0FB0EDB50776E71
:1062E00023D8B86EDECF02F0DDCF03F0040ED890D5
:1062F00002360336E804FBE1CF0EB7140210E85073
:10630000B76E060E7610766E0C0EB710B76E010ED5
:10631000006E020EE15C02E2E16AE552E16E0050BD
:10632000E552E7CFD9FF1200DECF00F0DDCF01F05C
:10633000D89001320032D890013200320050120061
:10634000D950FC0FE96EFF0EDA20EA6E12002DC064
:1063500032F02EC033F02FC034F030C035F01200D0
:10636000D9CFE6FFE1CFD9FF020EE126FE0EDB50CA
:106370001B0804E0FE0EDB50030823E1A3D8346AB7
:10638000356AAFD8F2EC26F0010A1BE0FA0EDBCF3B
:1063900004F0FB0EDBCF05F0FC0EDBCF06F0FD0EAC
:1063A000DBCF07F0326A336AA5D804C02DF005C0F0
:1063B0002EF006C02FF007C030F0E9EC26F0010AFD
:1063C00002E1000E73D0FA0EDBCF2DF0FB0EDBCF17
:1063D0002EF0FC0EDBCF2FF0FD0EDBCF30F0326A5B
:1063E000336A346A356AE2EC26F0010A02E1E66AB1
:1063F00009D068D87FD875D8E2EC26F0010A08E108
:10640000010EE66EFE0EDBCFE6FF21EC28F04CD04D
:10641000FA0EDBCF08F0FB0EDBCF09F0FC0EDBCF72
:106420000AF0FD0EDBCF0BF0326A336A63D808C086
:106430002DF009C02EF00AC02FF00BC030F0CCECCC
:1064400025F02DC004F02EC005F02FC006F030C09E
:1064500007F0326AC00E336E7F0E346E440E356E16
:106460001FEC26F02DC000F02EC001F02FC002F06E
:1064700030C003F0326A336A346A3F0E356E36EC50
:1064800025F0B3EC26F02EC0DEFF2FC0DDFF0F0E8F
:10649000E66EDECFE6FFDDCFE6FFFE0EDBCFE6FFEA
:1064A000B7EC30F0E552E552E552E552006E020ECF
:1064B000E15C02E2E16AE552E16E0050E552E7CFAD
:1064C000D9FF1200FA0EDBCF00F0FB0EDBCF01F09C
:1064D000FC0EDBCF02F0FD0EDBCF03F0326A336A35
:1064E000120000C02DF001C02EF002C02FF003C03A
:0E64F00030F01200A00E346E400E356E120019
:0264FE00D9CFF4
:10650000E6FFE1CFD9FF050EE126030EDB6A040E9C
:10651000DB6AB4D804E0FE0EDB50030873E1FE0E24
:10652000DBCFE6FF92EC2CF0E552F90EB16ECC0E0B
:10653000CD14DF6E310EDF10CD6EFE0E9D149D6EFC
:106540009DD80BE1FB0E9D149D6EFD0EDB5002E10C
:10655000040E01D0050E82D80AD0FE0EA314A36E3D
:10656000FD0EDB5002E1040E01D0050E7FD8BAEC1F
:1065700037F0C1EC37F0000907E0030EDB2A040E08
:1065800001E3DB2ABAEC37F05FD804E1FC0EDB5004
:10659000011838E073D803E1040E9E1407E1FE0EE3
:1065A000DB500308E6E1010EA414E3E0B36AB26A2B
:1065B00065D80BE1FB0E9D149D6EFD0EDB5002E1D4
:1065C000050E01D0040E4AD80AD0FE0EA314A36E05
:1065D000FD0EDB5002E1050E01D0040E47D8BAECE7
:1065E00037F0C1EC37F0000907E0030EDB2A040E98
:1065F00001E3DB2ABAEC37F027D807E1FC0EDB50C9
:10660000011803E1F36AF46A15D038D808E1040EE2
:106610009E1405E0BECFF3FFBFCFF4FF0BD0FE0EFC
:10662000DB500308DEE1010EA414DBE0B8CFF3FF7A
:10663000B9CFF4FF050EE15C02E2E16AE552E16EDA
:10664000E552E7CFD9FF1200030EDBCF00F0040EB6
:10665000DBCF01F0FB0EDB5000181200BD6EFB0E0D
:106660009E149E6E040E9D109D6E1200B76EFE0E5F
:10667000A414A46E010EA310A36E1200FE0EDB5034
:046680001B081200E1
:0C668400D9CFE6FFE1CFD9FF080EE126D8
:10669000060EDB6A070EDB6ADF6AABD80DE1DF06A8
:1066A000010EDFCFDBFFFC0EDB50100A21E0120AE7
:1066B00005E0080A03E052D0DF2AEFD792D8010E96
:1066C000DB50D880DF543FE394D82F0847E294D8BA
:1066D0003A0E005C43E28DD8D00F59D80A0EEC0276
:1066E000F3CFEDFFEF02F3CFEEFFF450ED26E7D747
:1066F00078D8010EDB50D880DF5425E37AD82F08F4
:1067000007E27AD83A0E005C03E273D8D00F13D0B8
:1067100070D8400807E270D8470E005C03E269D8E1
:10672000C90F09D066D8600819E266D8670E005C08
:1067300015E25FD8A90F2BD8040ED890EE36ED36AF
:10674000E806FBE1D6D7060EDBCF00F0070EDBCF65
:1067500001F000C0F3FF01C0F4FF02D0F36AF46A55
:10676000080EE15C02E2E16AE552E16EE552E7CF34
:10677000D9FF1200DF50E76EFD0EDBCFE9FFFE0E02
:10678000DBCFEAFFE750E926000EEA221200E66EB0
:10679000D950020FE96EDACFEAFFE552E750EE6E0C
:1067A000ED6A020EDBCF2EF0030EDBCF2FF0040ECE
:1067B000DBCF33F0050EDBCF34F0D6EC27F02DC065
:1067C00001F0D950060FE96EDACFEAFF2C50EE2621
:1067D0000150ED22DF06D950040FE96EDACFEAFF4F
:1067E0001200010EF36E040EF3CFDBFF050EDB6A21
:1067F0001200C0DFEF501200BDDFEFCF00F012003B
:10680000D9CFE6FFDACFE6FFFA0EE3CFD9FFFB0ED2
:10681000E3CFDAFFFC0EE3CFE9FFFD0EE3CFEAFFA3
:10682000E9CFF3FFEACFF4FFF80EE35003E1F90EEE
:10683000E35008E0F80EE30602E2F90EE306DECFCD
:10684000EEFFF2D7FF0EE3CFDAFFE552FF0EE3CF04
:10685000D9FFE5521200FB0EE3CFF6FFFC0EE3CFAB
:10686000F7FFFD0EE3CFF8FFFE0EE3CFE9FFFF0ECB
:10687000E3CFEAFFE9CFF3FFEACFF4FFF90EE350ED
:1068800003E1FA0EE35009E0F90EE30602E2FA0E24
:10689000E3060900F5CFEEFFF1D71200FE0EE3CFBD
:1068A000E9FFFF0EE3CFEAFFE9CFF3FFEACFF4FF02
:1068B000FB0EE35003E1FC0EE35009E0FB0EE306A0
:1068C00002E2FC0EE306FD0EE350EE6EF1D712007D
:1068D000D9CFE6FFDACFE6FFFA0EE3CFD9FFFB0E02
:1068E000E3CFDAFFFC0EE3CFE9FFFD0EE3CFEAFFD3
:1068F000DE50EF5C02E1EE66FBD7F36EFF0EE3CFF6
:10690000DAFFE552FF0EE3CFD9FFE552F350120054
:10691000FE0EE3CFE9FFFF0EE3CFEAFFF36AF46A6E
:10692000EE5203E0F34AF42AFBD71200FF0EE3CF46
:10693000F8FFE552FF0EE3CFF7FFE552FF0EE3CF7E
:10694000F6FFE552E66AE66AE66A0900F55209E0F2
:10695000FD0EE32A05E1FE0EE32A02E1FF0EE32A23
:10696000F4D7FD0EE3CF2DF0FE0EE3CF2EF0FF0E99
:06697000E3CF2FF012003E
:0A697600D9CFE6FFE1CFD9FF060EEE
:10698000E126FA0EDB5014E1010EE66EFE0EDBCFBF
:10699000E6FF21EC28F0E552E552DF6EE66AFE0ED6
:1069A000DBCFE6FF21EC28F0E552E552DF6E13D095
:1069B000E66AFE0EDBCFE6FF21EC28F0E552E55259
:1069C000DF6E010EE66EFE0EDBCFE6FF21EC28F057
:1069D000E552E552DF6EFB0EDB5031E1030EDB6A60
:1069E000040EDB6A030EDBCF00F0040EDBCF01F0F8
:1069F000030E005C000E015822E2010EDB6A020E5B
:106A0000DB6A010EDBCF00F0020EDBCF01F0FC0EE3
:106A1000DBCF02F0FD0EDBCF03F00250005C035031
:106A2000015807E20000010EDB2A020E01E3DB2A17
:106A3000E8D7030EDB2A040E01E3DB2AD3D7FB0ED3
:106A4000DB041CE1010EDB6A020EDB6A010EDBCF08
:106A500000F0020EDBCF01F0FC0EDBCF02F0FD0EEA
:106A6000DBCF03F00250005C0350015807E2000046
:106A7000010EDB2A020E01E3DB2AE8D7FA0EDB5017
:106A80000BE1010EE66EFE0EDBCFE6FF21EC28F0F7
:106A9000E552E552DF6E09D0E66AFE0EDBCFE6FF77
:106AA00021EC28F0E552E552DF6EDF5000D0006E99
:106AB000060EE15C02E2E16AE552E16E0050E55249
:066AC000E7CFD9FF120030
:0A6AC60041545A0D00415426460DBC
:106AD0000041542B42544D4F44452C6E0D004154FF
:106AE0002B425443414E43454C0D0041542B4254DC
:106AF0005343414E0D0041542B42545343414E2CBD
:106B00006E2C31323334350D0041542B42545343F3
:106B1000414E3131323233333434353536362C311F
:106B2000323334350D004154440D00415444313169
:106B3000323233333434353536360D004154480D56
:106B40000041542B42544C4153543F0D0041542BAF
:106B50004254525353492C300D0041542B42544B54
:106B600045593D224142434445464748494A4B4CDA
:106B70004D4E4F50220D0041542B425446502C6E26
:106B80000D0041542B42545345432C6E2C6D0D0087
:106B900041542B42544C504D2C6E0D0041542B420D
:106BA000544E414D453D22414243444546474849A4
:0E6BB0004A4B4C4D4E4F50220D0041540D00EB
:026BBE00D9CF2D
:106BC000E6FFE1CFD9FF030EE126020E4DD8010EFC
:106BD000EFCFDBFF030E48D8020EEFCFDBFF000E36
:106BE000E66EE66A010EDBCFE6FFFA0EDBCFE6FFCC
:106BF000FB0EDBCFE6FFFC0EDBCFE6FFFD0EDBCFAF
:106C0000E6FFFE0EDBCFE6FFE66A080EE66E9A0EA2
:106C1000E66E990EE66E190EE66E410EE66EE66AB7
:106C2000020EDBCFE6FFD2EC1AF0006E100EE15E32
:106C30000050DF6EDF50030A08E0070A06E0040A8E
:106C400002E0010A04E1DF5003D0DF0401D0000EAE
:106C5000006E030EE15C02E2E16AE552E16E005073
:106C6000E552E7CFD9FF1200E76EF80EDBCFE9FF60
:106C7000F90EDBCFEAFFE750E926000EEA22120008
:106C8000D9CFE6FFDACFE6FFE1CFD9FFE2CFDAFFD7
:106C9000E652E652E652E652D950F90F006EFF0E68
:106CA000DA20016E020E00C0DBFF030E01C0DBFF25
:106CB000020EDBCFE6FF030EDBCFE6FFF90EDBCFE4
:106CC000E6FFFA0EDBCFE6FFFB0EDBCFE6FFD95087
:106CD000FC0FE66EFF0EDA20E66ED7EC14F0006EC5
:106CE000070EE15C02E2E16AE552E16E0050F3CF8B
:106CF000DEFFF4CFDDFFFC0EDBCFE9FFFD0EDBCFC7
:106D0000EAFFEF6ADECF00F0DDCF01F000C0F3FF55
:106D100001C0F4FF040EE15C02E2E16AE552E16EBB
:0C6D2000E552E5CFDAFFE7CFD9FF120003
:046D2C00D9CFE6FFD6
:106D3000E1CFD9FF030EE12647D8010EEFCFDBFFED
:106D4000E76E42D8E750E926000EEA22020EEFCFA6
:106D5000DBFF010EDBCFE6FFFC0EDBCFE6FFFD0E17
:106D6000DBCFE6FFFE0EDBCFE6FF000EE66EE66A47
:106D7000E66A080EE66E000EE66EE66A9A0EE66EAB
:106D8000990EE66E190EE66E410EE66EE66A020E8A
:106D9000DBCFE6FF22EC04F0006E100EE15E005047
:106DA000DF6EDF5002E0010A02E1DF5001D0000E89
:106DB000006E030EE15C02E2E16AE552E16E005012
:106DC000E552E7CFD9FF1200FA0EDBCFE9FFFB0E49
:066DD000DBCFEAFF120018
:0A6DD6002A0EF66E080EF76E000E8E
:106DE000F86E00010900F550EB6F0900F550EC6FEB
:106DF00003E1EB6701D03DD00900F550E66F0900D3
:106E0000F550E76F0900F550E86F09000900F550EB
:106E1000E96E0900F550EA6E090009000900F55015
:106E2000E96F0900F550EA6F09000900F6CFEDF0AF
:106E3000F7CFEEF0F8CFEFF0E6C0F6FFE7C0F7FFD0
:106E4000E8C0F8FF0001E95302E1EA5307E0090056
:106E5000F550EE6EE907F8E2EA07F9D7EDC0F6FF64
:106E6000EEC0F7FFEFC0F8FF0001EB07000EEC5B90
:046E7000BFD7120076
:0C6E7400D9CFE6FFDACFE6FFE1CFD9FF6F
:106E8000E2CFDAFFFB0EDBCF00F0FC0EDBCF01F030
:106E90000001800E01141AE1FB0EDBCFE9FFFC0EAE
:106EA000DBCFEAFFEECFF3FFEDCFF4FFEE2A000ECB
:106EB000EF22F3CFE9FFF4CFEAFFFD0EDBCFEFFFC8
:106EC000EF50016AF36E01C0F4FF10D0FB0EDB50EF
:106ED000FE0806E1FD0EDBCFE6FF86EC38F005D0BC
:106EE000FD0EDBCFE6FFBCEC38F0E552E552E5CF16
:086EF000DAFFE7CFD9FF120021
:086EF800D9CFE6FFE1CFD9FF7D
:106F0000E652DF6A010EDF5C09E2000000000000CB
:106F10000000000000000000DF2AF4D7E552E5522F
:106F2000E7CFD9FF1200D9CFE6FFE1CFD9FF020E9C
:106F3000E126DE6ADD6ADECF00F0DDCF01F0FD0E76
:106F4000DBCF02F0FE0EDBCF03F00250005C0350FB
:106F5000015806E20000DF2A010E01E3DB2AEBD72D
:106F6000020EE15C02E2E16AE552E16EE552E7CF32
:046F7000D9FF120033
:0C6F7400450ED56E630ED66ED58EF294DD
:106F80001200F2A407D00001640EF76FE850D62675
:106F9000F294010C000CEEDFF4DF0009FDE01200BA
:106FA000D9CFE6FFE1CFD9FF020EE126DE6ADD6A26
:106FB000DECF00F0DDCF01F0FD0EDBCF02F0FE0EE4
:106FC000DBCF03F00250005C0350015806E2E3DF20
:106FD000DF2A010EEDE3DB2AEBD7020EE15C02E2D1
:0E6FE000E16AE552E16EE552E7CFD9FF1200FB
:026FEE002C5025
:106FF0003102F3CF28F0F4CF29F03202F3502926E2
:10700000000EF4202A6E2C503302F3502A26000E74
:10701000F4202B6E2C503402F3502B262D503102CD
:10702000F3502926F4502A22000E2B222D50320232
:10703000F3502A26F4502B222D503302F3502B26E6
:107040002E503102F3502A26F4502B222E503202B9
:0E705000F3502B262F503102F3502B26120046
:02705E002B6A9B
:107060002A6A296A286A200EE76ED8902C362D36B7
:107070002E362F36283629362A362B363150285CC4
:107080003250295833502A5834502B5809E3315084
:10709000285E3250295A33502A5A34502B5A2C2AFF
:0670A000E72EE4D7120008
:0A70A600D8CFE4FFE0CFE4FFE46E72
:1070B000DACFE4FFE2CFDAFFE652E552E5CFDAFFBE
:0C70C000E550E5CFE0FFE5CFD8FF100061
:0470CC00F36AF46A05
:1070D000FF0EE124E96EFF0EE220EA6EED6607D0B6
:1070E0002F0EEF6404D03A0EEF6001D0F32A1200A5
:1070F00016EE00F026EE00F0F86A379CEBEC36F066
:0C710000BDEC38F0E8EC0DF0FBD71200FD
:04710C00FF0EE3503F
:10711000ACBA04D0AF6AAB8EAC8A949CACA2FED75A
:08712000AD6EF36EF46A12007B
:08712800FF0EE350E84E1200D7
:0E713000000000D000D000D0E82EFAD71200E8
:02713E00DACFA6
:10714000E4FFE2CFDAFFE652E552E5CFDAFF1100C5
:1071500030313233343536373839616263646566CD
:01716000002E
:0E71620000EE00F00F0EEE6AEA62FDD712009A
:0871700025303458002575009C
:02717800120003
:02717A00120001
:04717C004242312E2C
:107180003068656C6C6F0124222321202B26022697
:06719000022602260200A7
:077196000D0A4F4B0D0A002A
:00000001FF
